******************************************************************************
            TI ARM Clang Linker PC v2.1.0                      
******************************************************************************
>> Linked Mon Nov 20 14:28:48 2023

OUTPUT FILE NAME:   <rfEasyLinkTx_433_CC1312R1_LAUNCHXL_tirtos7_ticlang.out>
ENTRY POINT SYMBOL: "ResetISR"  address: 00008d03


MEMORY CONFIGURATION

         name            origin    length      used     unused   attr    fill
----------------------  --------  ---------  --------  --------  ----  --------
  FLASH                 00000000   00058000  0000a33b  0004dcc5  R  X
  GPRAM                 11000000   00002000  00000000  00002000  RW X
  SRAM                  20000000   00014000  00005c1d  0000e3e3  RW X
  LOG_DATA              90000000   00040000  00000000  00040000  R   


SEGMENT ALLOCATION MAP

run origin  load origin   length   init length attrs members
----------  ----------- ---------- ----------- ----- -------
00000000    00000000    0000a123   0000a123    r-x
  00000000    00000000    0000003c   0000003c    r-- .resetVecs
  0000003c    0000003c    00008d50   00008d50    r-x .text
  00008d8c    00008d8c    00001397   00001397    r-- .rodata
0000a124    0000a124    00000008   00000008    rw-
  0000a124    0000a124    00000008   00000008    rw- .args
0000a12c    0000a12c    000001b8   000001b8    r--
  0000a12c    0000a12c    000001b8   000001b8    r-- .cinit
00057fa8    00057fa8    00000058   00000058    r--
  00057fa8    00057fa8    00000058   00000058    r-- .ccfg
200000d8    200000d8    00004000   00000000    r--
  200000d8    200000d8    00004000   00000000    r-- .priheap
200040d8    200040d8    00001745   00000000    rw-
  200040d8    200040d8    000010e8   00000000    rw- .bss
  200051c0    200051c0    0000065d   00000000    rw- .data
20013c00    20013c00    00000400   00000000    rw-
  20013c00    20013c00    00000400   00000000    rw- .stack


SECTION ALLOCATION MAP

 output                                  attributes/
section   page    origin      length       input sections
--------  ----  ----------  ----------   ----------------
.binit     0    00000000    00000000     

.cinit     0    0000a12c    000001b8     
                  0000a12c    00000194     (.cinit..data.load) [load image, compression = lzss]
                  0000a2c0    0000000c     (__TI_handler_table)
                  0000a2cc    00000008     (.cinit..bss.load) [load image, compression = zero_init]
                  0000a2d4    00000010     (__TI_cinit_table)

.init_array 
*          0    00000000    00000000     UNINITIALIZED

.ccfg      0    00057fa8    00000058     
                  00057fa8    00000058     ti_devices_config.o (.ccfg)

.bss       0    200040d8    000010e8     UNINITIALIZED
                  200040d8    00000400     rfEasyLinkTx.o (.bss.txTaskStack)
                  200044d8    000002c0     rf_multiMode_cc13x2.a : RFCC26X2_multiMode.c.cc13x2.ticlang.o (.bss.RF_cmdPool)
                  20004798    00000200     (.common:ti_sysbios_knl_Idle_taskStack)
                  20004998    00000100     EasyLink.o (.bss.rfObject)
                  20004a98    000000d8     (.common:ti_sysbios_family_arm_m3_Hwi_dispatchTable)
                  20004b70    0000008a     EasyLink.o (.bss.txBuffer)
                  20004bfa    00000002     rfEasyLinkTx.o (.bss.seqNumber)
                  20004bfc    0000007c     (.common:gpioCallbackFunctions)
                  20004c78    0000007c     (.common:gpioUserArgs)
                  20004cf4    00000004     EasyLink.o (.bss.busyMutex)
                  20004cf8    00000068     rf_multiMode_cc13x2.a : RFCC26X2_multiMode.c.cc13x2.ticlang.o (.bss.RF_ratModule)
                  20004d60    00000060     (.common:ti_sysbios_knl_ClockSupport_timerStruct)
                  20004dc0    00000058     (.common:ti_sysbios_knl_Idle_taskStruct)
                  20004e18    00000058     (.common:txTask)
                  20004e70    00000044                           : RFCC26X2_multiMode.c.cc13x2.ticlang.o (.bss.RF_clkInactivityObj)
                  20004eb4    00000044                           : RFCC26X2_multiMode.c.cc13x2.ticlang.o (.bss.RF_clkPowerUpObj)
                  20004ef8    0000003c                           : RFCC26X2_multiMode.c.cc13x2.ticlang.o (.bss.RF_swiHwObj)
                  20004f34    00000030     EasyLink.o (.bss.EasyLink_cmdPropRxAdv)
                  20004f64    00000030     (.common:ti_sysbios_knl_Swi_readyQs)
                  20004f94    00000030     (.common:ti_sysbios_knl_Task_readyQs)
                  20004fc4    0000002c     (.common:BIOS_heapMemObject)
                  20004ff0    00000028     EasyLink.o (.bss.EasyLink_cmdPropRadioSetup)
                  20005018    00000028     (.common:BIOS_rtsGate)
                  20005040    00000028     (.common:ti_sysbios_heaps_HeapMem_gate)
                  20005068    00000024     rfEasyLinkTx.o (.bss.txTaskParams)
                  2000508c    00000020     EasyLink.o (.bss.EasyLink_cmdPropTxAdv)
                  200050ac    00000020     EasyLink.o (.bss.rfParams)
                  200050cc    00000020     EasyLink.o (.bss.schParams_prop)
                  200050ec    00000020     (.common:ti_sysbios_runtime_System_atexitHandlers)
                  2000510c    0000001c     EasyLink.o (.bss.EasyLink_cmdPropCs)
                  20005128    0000001c     drivers_cc13x2.a : GPIOCC26X2.c.obj (.bss.gpioHwi)
                  20005144    00000018     EasyLink.o (.bss.EasyLink_cmdFs)
                  2000515c    00000010     EasyLink.o (.bss.EasyLink_RF_prop)
                  2000516c    00000010     EasyLink.o (.bss.EasyLink_params)
                  2000517c    0000000c     EasyLink.o (.bss.rxStatistics)
                  20005188    00000008     EasyLink.o (.bss.dataQueue)
                  20005190    00000004     EasyLink.o (.bss.getRN)
                  20005194    00000004     driverlib.lib : osc.o (.bss.oscHfGlobals.0)
                  20005198    00000004                   : osc.o (.bss.oscHfGlobals.2)
                  2000519c    00000004                   : osc.o (.bss.oscHfGlobals.3)
                  200051a0    00000004                   : osc.o (.bss.oscHfGlobals.4)
                  200051a4    00000004     EasyLink.o (.bss.rfHandle)
                  200051a8    00000004     EasyLink.o (.bss.txCb)
                  200051ac    00000004     rfEasyLinkTx.o (.bss.txDoneSem)
                  200051b0    00000004     (.common:PowerCC26XX_swiKey)
                  200051b4    00000004     (.common:PowerCC26XX_taskKey)
                  200051b8    00000004     (.common:ti_sysbios_family_arm_cc26xx_TimestampProvider_Module_state)
                  200051bc    00000004     (.common:ti_sysbios_knl_Task_defaultStackHeap)

.data      0    200051c0    0000065d     UNINITIALIZED
                  200051c0    00000174     drivers_cc13x2.a : PowerCC26X2.c.obj (.data.PowerCC26X2_module)
                  20005334    0000007c     ti_drivers_config.o (.data.gpioPinConfigs)
                  200053b0    00000068     rf_multiMode_cc13x2.a : RFCC26X2_multiMode.c.cc13x2.ticlang.o (.data..L_MergedGlobals.1)
                  20005418    00000068     ti_sysbios_config.o (.data.ti_sysbios_knl_Clock_Module_state)
                  20005480    00000064     rf_multiMode_cc13x2.a : RFCC26X2_multiMode.c.cc13x2.ticlang.o (.data..L_MergedGlobals.3)
                  200054e4    00000064     ti_radio_config.o (.data.txPowerTable_433_pa13)
                  20005548    00000058     rf_multiMode_cc13x2.a : RFCC26X2_multiMode.c.cc13x2.ticlang.o (.data..L_MergedGlobals.2)
                  200055a0    00000040     EasyLink.o (.data.addrFilterTable)
                  200055e0    0000003c     ti_sysbios_config.o (.data.ti_sysbios_family_arm_m3_Hwi_Module_state)
                  2000561c    0000003c     ti_sysbios_config.o (.data.ti_sysbios_knl_Task_Module_state)
                  20005658    00000030     ti_radio_config.o (.data.RF_cmdPropRxAdv)
                  20005688    0000002c     ti_sysbios_config.o (.data.BIOS_Module_state)
                  200056b4    00000028     ti_radio_config.o (.data.RF_cmdPropRadioDivSetup)
                  200056dc    00000028     ti_radio_config.o (.data.pOverrides)
                  20005704    00000028     ti_sysbios_config.o (.data.ti_sysbios_knl_Swi_Module_state)
                  2000572c    00000024     ti_easylink_config.o (.data.EasyLink_supportedPhys)
                  20005750    00000018     ti_radio_config.o (.data.RF_cmdFs)
                  20005768    00000018     ti_radio_config.o (.data.RF_cmdPropTx)
                  20005780    00000010     ti_radio_config.o (.data.RF_prop)
                  20005790    00000010     driverlib.lib : osc.o (.data._hposcCoeffs)
                  200057a0    0000000c     ti_sysbios_config.o (.data.ti_sysbios_family_arm_cc26xx_Timer_Module_state)
                  200057ac    0000000c     ti_sysbios_config.o (.data.ti_sysbios_runtime_Error_ignore)
                  200057b8    0000000c     ti_sysbios_config.o (.data.ti_sysbios_runtime_System_Module_state)
                  200057c4    00000008     rf_multiMode_cc13x2.a : RFCC26X2_multiMode.c.cc13x2.ticlang.o (.data..L_MergedGlobals)
                  200057cc    00000008                           : RFCC26X2_multiMode.c.cc13x2.ticlang.o (.data.RFCC26XX_schedulerPolicy)
                  200057d4    00000008     ti_sysbios_config.o (.data.ti_sysbios_gates_GateMutex_Module_state)
                  200057dc    00000008     ti_sysbios_config.o (.data.ti_sysbios_heaps_HeapMem_Module_state)
                  200057e4    00000008     ti_sysbios_config.o (.data.ti_sysbios_knl_Semaphore_Module_state)
                  200057ec    00000004     rf_multiMode_cc13x2.a : RFCC26X2_multiMode.c.cc13x2.ticlang.o (.data.RF_fsmActiveState.lfClockSourceLast)
                  200057f0    00000004     libc.a : _lock.c.obj (.data._lock)
                  200057f4    00000004            : _lock.c.obj (.data._unlock)
                  200057f8    00000004     EasyLink.o (.data.cmdPriority)
                  200057fc    00000004     EasyLink.o (.data.inactivityTimeout)
                  20005800    00000004     libc.a : rand.c.obj (.data.next)
                  20005804    00000004     EasyLink.o (.data.rfSetting)
                  20005808    00000004     ti_sysbios_config.o (.data.terminatedList)
                  2000580c    00000004     ti_sysbios_config.o (.data.ti_sysbios_runtime_Memory_defaultHeapInstance)
                  20005810    00000002     EasyLink.o (.data.asyncCmdHndl)
                  20005812    00000001     EasyLink.o (.data.addrSize)
                  20005813    00000001     rf_multiMode_cc13x2.a : rf_patch_cpe_multi_protocol.c.cc13x2.ticlang.o (.data.bMultiProtocolPatchEntered)
                  20005814    00000001     EasyLink.o (.data.configured)
                  20005815    00000001     EasyLink.o (.data.hdrSize)
                  20005816    00000001     drivers_cc13x2.a : GPIOCC26X2.c.obj (.data.initCalled)
                  20005817    00000001     EasyLink.o (.data.rfModeMultiClient)
                  20005818    00000001     EasyLink.o (.data.rfParamsConfigured)
                  20005819    00000001     EasyLink.o (.data.suspended)
                  2000581a    00000001     ti_sysbios_config.o (.data.ti_sysbios_knl_Idle_initDone)
                  2000581b    00000001     ti_sysbios_config.o (.data.ti_sysbios_runtime_Startup_done)
                  2000581c    00000001     EasyLink.o (.data.useIeeeHeader)

.stack     0    20013c00    00000400     UNINITIALIZED
                  20013c00    00000004     sysbios.a : boot_cortex_m.obj (.stack)
                  20013c04    000003fc     --HOLE--

.priheap   0    200000d8    00004000     UNINITIALIZED
                  200000d8    00004000     --HOLE--

.log_data 
*          0    90000000    00000000     COPY SECTION

.resetVecs 
*          0    00000000    0000003c     
                  00000000    0000003c     ti_sysbios_config.o (.resetVecs)

.vecs      0    20000000    000000d8     NOLOAD SECTION
                  20000000    000000d8     ti_sysbios_config.o (.vecs)

__llvm_prf_cnts 
*          0    20000000    00000000     UNINITIALIZED

__llvm_prf_bits 
*          0    20000000    00000000     UNINITIALIZED

.text      0    0000003c    00008d50     
                  0000003c    00000842     EasyLink.o (.text.EasyLink_init)
                  0000087e    00000002     ti_sysbios_config.o (.text.BIOS_nullFunc)
                  00000880    00000498     rf_multiMode_cc13x2.a : RFCC26X2_multiMode.c.cc13x2.ticlang.o (.text.RF_fsmActiveState)
                  00000d18    000002fe     EasyLink.o (.text.EasyLink_transmitAsync)
                  00001016    00000002     ti_drivers_config.o (.text.Board_initHook)
                  00001018    0000029c     rf_multiMode_cc13x2.a : RFCC26X2_multiMode.c.cc13x2.ticlang.o (.text.RF_open)
                  000012b4    000001fa     ti_sysbios_config.o (.text.ti_sysbios_family_arm_m3_Hwi_excFillContext)
                  000014ae    00000002     rf_multiMode_cc13x2.a : rfc.c.cc13x2.ticlang.o (.text.NOROM_RFCCpePatchReset)
                  000014b0    000001e4                           : RFCC26X2_multiMode.c.cc13x2.ticlang.o (.text.RF_scheduleCmd)
                  00001694    000001e0                           : RFCC26X2_multiMode.c.cc13x2.ticlang.o (.text.RF_dispatchNextCmd)
                  00001874    000001aa     ti_sysbios_config.o (.text.ti_sysbios_knl_TaskSupport_buildTaskStack)
                  00001a1e    00000198     ti_sysbios_config.o (.text.ti_sysbios_family_arm_cc26xx_Timer_construct)
                  00001bb6    00000002     rf_multiMode_cc13x2.a : RFCC26X2_multiMode.c.cc13x2.ticlang.o (.text.RF_defaultCallback)
                  00001bb8    00000194     drivers_cc13x2.a : PowerCC26X2_calibrateRCOSC.c.obj (.text.PowerCC26X2_auxISR)
                  00001d4c    0000018e     ti_sysbios_config.o (.text.ti_sysbios_knl_Task_Instance_init)
                  00001eda    0000015e     rfEasyLinkTx.o (.text.rfEasyLinkTxFnx)
                  00002038    0000015c     drivers_cc13x2.a : PowerCC26X2.c.obj (.text.Power_sleep)
                  00002194    0000013e     ti_sysbios_config.o (.text.PowerCC26XX_standbyPolicy)
                  000022d2    0000013e     ti_sysbios_config.o (.text.ti_sysbios_heaps_HeapMem_allocUnprotected)
                  00002410    0000013c     rf_multiMode_cc13x2.a : RFCC26X2_multiMode.c.cc13x2.ticlang.o (.text.RF_radioOpDoneCb)
                  0000254c    0000013c     ti_sysbios_config.o (.text.ti_sysbios_knl_Clock_workFuncDynamic)
                  00002688    0000012c     rf_multiMode_cc13x2.a : RFCC26X2_multiMode.c.cc13x2.ticlang.o (.text.RF_close)
                  000027b4    0000012c                           : RFCC26X2_multiMode.c.cc13x2.ticlang.o (.text.RF_fsmSetupState)
                  000028e0    00000124                           : RFCC26X2_multiMode.c.cc13x2.ticlang.o (.text.RF_abortCmd)
                  00002a04    0000011c     sysbios.a : Hwi_asm_gnu.obj (.text.ti_sysbios_family_arm_m3_Hwi_dispatch)
                  00002b20    00000118     drivers_cc13x2.a : PowerCC26X2.c.obj (.text.Power_init)
                  00002c38    00000118     rf_multiMode_cc13x2.a : RFCC26X2_multiMode.c.cc13x2.ticlang.o (.text.RF_decodeOverridePointers)
                  00002d50    0000010e     ti_sysbios_config.o (.text.ti_sysbios_knl_Semaphore_pend)
                  00002e5e    00000002     libclang_rt.builtins.a : aeabi_div0.c.obj (.text.__aeabi_ldiv0)
                  00002e60    0000010c     drivers_cc13x2.a : PowerCC26X2_calibrateRCOSC.c.obj (.text.PowerCC26X2_calibrate)
                  00002f6c    0000010a     ti_sysbios_config.o (.text.ti_sysbios_knl_Task_Instance_finalize)
                  00003076    00000002     libc.a : _lock.c.obj (.text._nop)
                  00003078    00000108     rf_multiMode_cc13x2.a : RFCC26X2_multiMode.c.cc13x2.ticlang.o (.text.RF_fsmPowerUpState)
                  00003180    00000104     drivers_cc13x2.a : GPIOCC26X2.c.obj (.text.GPIO_init)
                  00003284    000000fe     ti_sysbios_config.o (.text.ti_sysbios_family_arm_m3_Hwi_Instance_init)
                  00003382    00000002     drivers_cc13x2.a : PowerCC26X2.c.obj (.text.emptyClockFunc)
                  00003384    000000fc     rf_multiMode_cc13x2.a : RFCC26X2_multiMode.c.cc13x2.ticlang.o (.text.RF_hwiCpe0Active)
                  00003480    000000f4     driverlib.lib : sys_ctrl.o (.text.NOROM_SysCtrlStandby)
                  00003574    000000ee     ti_sysbios_config.o (.text.ti_sysbios_knl_Clock_startI)
                  00003662    000000e4     ti_sysbios_config.o (.text.ti_sysbios_family_arm_m3_Hwi_initNVIC)
                  00003746    000000dc     EasyLink.o (.text.EasyLink_abort)
                  00003822    000000dc     ti_sysbios_config.o (.text.ti_sysbios_knl_Task_checkStacks)
                  000038fe    000000da     ti_sysbios_config.o (.text.ti_sysbios_heaps_HeapMem_freeUnprotected)
                  000039d8    000000d0     drivers_cc13x2.a : PowerCC26X2.c.obj (.text.configureXOSCHF)
                  00003aa8    000000cc     rf_multiMode_cc13x2.a : RFCC26X2_multiMode.c.cc13x2.ticlang.o (.text.RF_postCmd)
                  00003b74    000000ca                           : RFCC26X2_multiMode.c.cc13x2.ticlang.o (.text.RF_updatePaConfiguration)
                  00003c3e    00000002     ti_sysbios_config.o (.text.ti_sysbios_family_arm_cc26xx_Timer_startup)
                  00003c40    000000c4     driverlib.lib : setup.o (.text.NOROM_SetupTrimDevice)
                  00003d04    000000c4                   : setup.o (.text.TrimAfterColdResetWakeupFromShutDown)
                  00003dc8    000000c0     ti_sysbios_config.o (.text.ti_sysbios_knl_Clock_walkQueueDynamic)
                  00003e88    000000c0     ti_sysbios_config.o (.text.ti_sysbios_knl_Swi_restoreHwi)
                  00003f48    000000bc     rf_multiMode_cc13x2.a : RFCC26X2_multiMode.c.cc13x2.ticlang.o (.text.RF_swiHw)
                  00004004    000000bc     ti_sysbios_config.o (.text.ti_sysbios_knl_Task_postInit)
                  000040c0    000000b8     ti_sysbios_config.o (.text.ti_sysbios_knl_Swi_Instance_init)
                  00004178    000000b4     driverlib.lib : osc.o (.text.NOROM_OSCHF_AttemptToSwitchToXosc)
                  0000422c    000000b4     drivers_cc13x2.a : PowerCC26X2.c.obj (.text.Power_releaseDependency)
                  000042e0    000000b0                      : PowerCC26X2.c.obj (.text.Power_setDependency)
                  00004390    000000b0     libclang_rt.builtins.a : udivmoddi4.S.obj (.text)
                  00004440    000000ae     EasyLink.o (.text.txDoneCallback)
                  000044ee    00000002     ti_sysbios_config.o (.text.ti_sysbios_knl_TaskSupport_init)
                  000044f0    000000ac     rf_multiMode_cc13x2.a : RFCC26X2_multiMode.c.cc13x2.ticlang.o (.text.RF_initRadioSetup)
                  0000459c    000000ac                           : RFCC26X2_multiMode.c.cc13x2.ticlang.o (.text.RF_pendCmd)
                  00004648    000000aa     driverlib.lib : chipinfo.o (.text.NOROM_ChipInfo_GetChipType)
                  000046f2    000000a2     ti_sysbios_config.o (.text.ti_sysbios_knl_TaskSupport_start)
                  00004794    000000a2     ti_sysbios_config.o (.text.ti_sysbios_knl_Task_schedule)
                  00004836    00000002     ti_sysbios_config.o (.text.ti_sysbios_runtime_SysCallback_defaultInit)
                  00004838    000000a0     rf_multiMode_cc13x2.a : RFCC26X2_multiMode.c.cc13x2.ticlang.o (.text.RF_calculateDispatchTime)
                  000048d8    0000009a                           : RFCC26X2_multiMode.c.cc13x2.ticlang.o (.text.RF_defaultSubmitPolicy)
                  00004972    00000098     EasyLink.o (.text.calculateCmdTime)
                  00004a0a    00000096     rf_multiMode_cc13x2.a : RFCC26X2_multiMode.c.cc13x2.ticlang.o (.text.RF_verifyGap)
                  00004aa0    00000094                           : RFCC26X2_multiMode.c.cc13x2.ticlang.o (.text.RF_ratRestartChannels)
                  00004b34    00000094     ti_sysbios_config.o (.text.ti_sysbios_heaps_HeapMem_Instance_init)
                  00004bc8    0000008e     ti_sysbios_config.o (.text.ti_sysbios_family_arm_m3_Hwi_excHandlerMin)
                  00004c56    0000008e     ti_sysbios_config.o (.text.ti_sysbios_knl_Swi_runLoop)
                  00004ce4    0000008c     drivers_cc13x2.a : GPIOCC26XX.c.obj (.text.GPIO_setConfig)
                  00004d70    0000008c     ti_sysbios_config.o (.text.ti_sysbios_family_arm_m3_Hwi_construct2)
                  00004dfc    0000008a     ti_sysbios_config.o (.text.ti_sysbios_knl_Semaphore_post)
                  00004e86    00000002     --HOLE-- [fill = 0]
                  00004e88    00000088     rf_multiMode_cc13x2.a : RFCC26X2_multiMode.c.cc13x2.ticlang.o (.text.RF_cmdDispatchTime)
                  00004f10    00000088                           : RFCC26X2_multiMode.c.cc13x2.ticlang.o (.text.RF_discardPendCmd)
                  00004f98    00000088     ti_sysbios_config.o (.text.ti_sysbios_family_arm_m3_Hwi_postInit)
                  00005020    00000086     ti_sysbios_config.o (.text.ti_sysbios_runtime_Memory_alloc)
                  000050a6    00000084     ti_sysbios_config.o (.text.ti_sysbios_knl_Task_startup)
                  0000512a    00000082     ti_sysbios_config.o (.text.ti_sysbios_family_arm_m3_Hwi_getStackInfo)
                  000051ac    00000080     driverlib.lib : sys_ctrl.o (.text.NOROM_SysCtrlSetRechargeBeforePowerDown)
                  0000522c    0000007e     ti_drivers_config.o (.text.Board_sendExtFlashByte)
                  000052aa    0000007c     ti_sysbios_config.o (.text.SwiP_construct)
                  00005326    0000007c     ti_sysbios_config.o (.text.ti_sysbios_family_arm_cc26xx_Timer_periodicStub)
                  000053a2    0000007c     ti_sysbios_config.o (.text.ti_sysbios_knl_Swi_schedule)
                  0000541e    0000007a     EasyLink.o (.text.createTxAdvFromTx)
                  00005498    0000007a     ti_sysbios_config.o (.text.ti_sysbios_family_arm_m3_Hwi_dispatchC)
                  00005512    0000007a     ti_sysbios_config.o (.text.ti_sysbios_knl_Idle_init)
                  0000558c    00000078     driverlib.lib : osc.o (.text.NOROM_OSCHF_SwitchToRcOscTurnOffXosc)
                  00005604    00000078                   : osc.o (.text.NOROM_OSC_CapArrayAdjustWorkaround_Boot)
                  0000567c    00000078     drivers_cc13x2.a : PowerCC26X2_calibrateRCOSC_helpers.c.obj (.text.PowerCC26X2_updateSubSecInc)
                  000056f4    00000078     rf_multiMode_cc13x2.a : RFCC26X2_multiMode.c.cc13x2.ticlang.o (.text.RF_ratFreeChannel)
                  0000576c    00000078     ti_sysbios_config.o (.text.ti_sysbios_family_arm_m3_Hwi_disableInterrupt)
                  000057e4    00000078     ti_sysbios_config.o (.text.ti_sysbios_knl_Swi_run)
                  0000585c    00000078     ti_sysbios_config.o (.text.ti_sysbios_knl_Task_blockI)
                  000058d4    00000074     rf_multiMode_cc13x2.a : RFCC26X2_multiMode.c.cc13x2.ticlang.o (.text.RF_hwiHw)
                  00005948    00000074     ti_sysbios_config.o (.text.ti_sysbios_heaps_HeapMem_getStats)
                  000059bc    00000072     ti_sysbios_config.o (.text.ti_sysbios_family_arm_cc26xx_Timer_setThreshold)
                  00005a2e    00000070     ti_sysbios_config.o (.text.ti_sysbios_family_arm_m3_Hwi_enableInterrupt)
                  00005a9e    0000006e     ti_sysbios_config.o (.text.BIOS_init)
                  00005b0c    0000006e     ti_drivers_config.o (.text.Board_shutDownExtFlash)
                  00005b7a    0000006e     ti_sysbios_config.o (.text.ti_sysbios_knl_Clock_init)
                  00005be8    0000006c     rf_multiMode_cc13x2.a : RFCC26X2_multiMode.c.cc13x2.ticlang.o (.text.RF_issueRadioFreeCb)
                  00005c54    0000006c                           : rf_patch_cpe_multi_protocol.c.cc13x2.ticlang.o (.text.configureMultiProtocolPatch)
                  00005cc0    0000006a                           : RFCC26X2_multiMode.c.cc13x2.ticlang.o (.text.RF_detachOverrides)
                  00005d2a    0000006a     libc.a : copy_decompress_lzss.c.obj (.text:decompress:lzss)
                  00005d94    00000066     rf_multiMode_cc13x2.a : RFCC26X2_multiMode.c.cc13x2.ticlang.o (.text.RF_attachOverrides)
                  00005dfa    00000066     ti_sysbios_config.o (.text.ti_sysbios_family_arm_cc26xx_Timer_start)
                  00005e60    00000066     ti_sysbios_config.o (.text.ti_sysbios_family_arm_m3_Hwi_Instance_finalize)
                  00005ec6    00000002     --HOLE-- [fill = 0]
                  00005ec8    00000064     drivers_cc13x2.a : PowerCC26X2_calibrateRCOSC.c.obj (.text.PowerCC26X2_initiateCalibration)
                  00005f2c    00000064     rf_multiMode_cc13x2.a : RFCC26X2_multiMode.c.cc13x2.ticlang.o (.text.RF_dispatchNextEvent)
                  00005f90    00000064                           : RFCC26X2_multiMode.c.cc13x2.ticlang.o (.text.RF_hwiCpe0PowerFsm)
                  00005ff4    00000062                           : RFCC26X2_multiMode.c.cc13x2.ticlang.o (.text.RF_syncCb)
                  00006056    00000060     ti_sysbios_config.o (.text.ti_sysbios_knl_ClockSupport_init)
                  000060b6    00000002     --HOLE-- [fill = 0]
                  000060b8    0000005e     rf_multiMode_cc13x2.a : rfc.c.cc13x2.ticlang.o (.text.NOROM_RFCAnaDivTxOverride)
                  00006116    0000005e     ti_sysbios_config.o (.text.ti_sysbios_knl_Swi_post)
                  00006174    0000005c     ti_sysbios_config.o (.text.ClockP_construct)
                  000061d0    0000005c     ti_sysbios_config.o (.text.ti_sysbios_heaps_HeapMem_alloc)
                  0000622c    0000005c     ti_sysbios_config.o (.text.ti_sysbios_knl_Task_init)
                  00006288    00000058     ti_sysbios_config.o (.text.AONRTCEventClear)
                  000062e0    00000058     ti_sysbios_config.o (.text.HwiP_construct)
                  00006338    00000058     rf_multiMode_cc13x2.a : RFCC26X2_multiMode.c.cc13x2.ticlang.o (.text.RF_applyRfCorePatch)
                  00006390    00000058     ti_sysbios_config.o (.text.ti_sysbios_family_arm_m3_Hwi_construct)
                  000063e8    00000058     sysbios.a : Hwi_asm_switch_gnu.obj (.text.ti_sysbios_family_arm_m3_Hwi_initStacks)
                  00006440    00000058     ti_sysbios_config.o (.text.ti_sysbios_heaps_HeapMem_construct)
                  00006498    00000058     ti_sysbios_config.o (.text.ti_sysbios_knl_Swi_init)
                  000064f0    00000056     ti_sysbios_config.o (.text.AONRTCCompareValueSet)
                  00006546    00000056     ti_sysbios_config.o (.text.ti_sysbios_family_arm_cc26xx_Timer_getCurrentTick)
                  0000659c    00000056     ti_sysbios_config.o (.text.ti_sysbios_knl_Clock_Instance_init)
                  000065f2    00000056     ti_sysbios_config.o (.text.ti_sysbios_runtime_System_atexit)
                  00006648    00000054     ti_sysbios_config.o (.text.AONRTCChannelEnable)
                  0000669c    00000054     ti_sysbios_config.o (.text.BIOS_startFunc)
                  000066f0    00000054     rf_multiMode_cc13x2.a : RFCC26X2_multiMode.c.cc13x2.ticlang.o (.text.RF_fsmXOSCState)
                  00006744    00000054                           : RFCC26X2_multiMode.c.cc13x2.ticlang.o (.text.RF_getCurrentTime)
                  00006798    00000052     driverlib.lib : chipinfo.o (.text.NOROM_ChipInfo_GetHwRevision)
                  000067ea    00000002     --HOLE-- [fill = 0]
                  000067ec    00000050     rf_multiMode_cc13x2.a : RFCC26X2_multiMode.c.cc13x2.ticlang.o (.text.RF_wakeupNotification)
                  0000683c    00000050     ti_sysbios_config.o (.text.ti_sysbios_family_arm_cc26xx_Timer_setNextTick)
                  0000688c    0000004e     ti_sysbios_config.o (.text.ti_sysbios_knl_Swi_restore)
                  000068da    0000004c     driverlib.lib : osc.o (.text.NOROM_OSC_HPOSCRelativeFrequencyOffsetGet)
                  00006926    0000004c     rfEasyLinkTx.o (.text.main)
                  00006972    00000002     --HOLE-- [fill = 0]
                  00006974    0000004c     drivers_cc13x2.a : PowerCC26X2.c.obj (.text.switchXOSCHF)
                  000069c0    0000004c     ti_sysbios_config.o (.text.ti_sysbios_knl_Clock_getTimeout)
                  00006a0c    0000004c     ti_sysbios_config.o (.text.ti_sysbios_runtime_System_processAtExit)
                  00006a58    0000004c     rfEasyLinkTx.o (.text.txDoneCb)
                  00006aa4    0000004c     rfEasyLinkTx.o (.text.txTask_init)
                  00006af0    0000004a     ti_sysbios_config.o (.text.ti_sysbios_knl_Task_construct)
                  00006b3a    00000002     --HOLE-- [fill = 0]
                  00006b3c    00000048     driverlib.lib : aux_sysif.o (.text.NOROM_AUXSYSIFOpModeChange)
                  00006b84    00000048     rf_multiMode_cc13x2.a : rfc.c.cc13x2.ticlang.o (.text.NOROM_RFCSynthPowerDown)
                  00006bcc    00000048     drivers_cc13x2.a : PowerCC26X2.c.obj (.text.PowerCC26XX_switchXOSC_HF)
                  00006c14    00000048                      : PowerCC26X2.c.obj (.text.oscillatorISR)
                  00006c5c    00000048     ti_sysbios_config.o (.text.ti_sysbios_family_arm_m3_Hwi_init)
                  00006ca4    00000046     ti_sysbios_config.o (.text.ti_sysbios_knl_Semaphore_Instance_init)
                  00006cea    00000046     ti_sysbios_config.o (.text.ti_sysbios_knl_Swi_construct)
                  00006d30    00000046     ti_sysbios_config.o (.text.ti_sysbios_knl_Task_processVitalTaskFlag)
                  00006d76    00000046     ti_sysbios_config.o (.text.ti_sysbios_knl_Task_unblockI)
                  00006dbc    00000044     ti_sysbios_config.o (.text.BIOS_rtsLock)
                  00006e00    00000044     drivers_cc13x2.a : GPIOCC26X2.c.obj (.text.GPIO_hwiIntFxn)
                  00006e44    00000044     driverlib.lib : prcm.o (.text.NOROM_PRCMPowerDomainsAllOff)
                  00006e88    00000044                   : prcm.o (.text.NOROM_PRCMPowerDomainsAllOn)
                  00006ecc    00000044     drivers_cc13x2.a : PowerCC26X2.c.obj (.text.PowerCC26XX_isStableXOSC_HF)
                  00006f10    00000044     rf_multiMode_cc13x2.a : RFCC26X2_multiMode.c.cc13x2.ticlang.o (.text.RF_cmdGet)
                  00006f54    00000044                           : RFCC26X2_multiMode.c.cc13x2.ticlang.o (.text.RF_updatePowerupDuration)
                  00006f98    00000044     ti_sysbios_config.o (.text._pthread_cleanupFxn)
                  00006fdc    00000044     ti_sysbios_config.o (.text.ti_sysbios_knl_Task_restore)
                  00007020    00000044     ti_sysbios_config.o (.text.ti_sysbios_runtime_Error_raiseX)
                  00007064    00000042     EasyLink.o (.text.EasyLink_getAbsTime)
                  000070a6    00000002     --HOLE-- [fill = 0]
                  000070a8    00000040     drivers_cc13x2.a : PowerCC26X2_calibrateRCOSC.c.obj (.text.PowerCC26X2_RCOSC_clockFunc)
                  000070e8    00000040                      : PowerCC26X2_calibrateRCOSC_helpers.c.obj (.text.PowerCC26X2_setAclkRefSrc)
                  00007128    00000040     ti_sysbios_config.o (.text.ti_sysbios_gates_GateMutex_enter)
                  00007168    00000040     ti_sysbios_config.o (.text.ti_sysbios_knl_Semaphore_pendTimeout)
                  000071a8    00000040     ti_sysbios_config.o (.text.ti_sysbios_knl_Task_exit)
                  000071e8    0000003e     ti_sysbios_config.o (.text.ti_sysbios_knl_Clock_getTicksUntilInterrupt)
                  00007226    0000003c     ti_sysbios_config.o (.text.BIOS_atExitFunc)
                  00007262    00000002     --HOLE-- [fill = 0]
                  00007264    0000003c     drivers_cc13x2.a : GPIO.c.obj (.text.GPIO_resetConfig)
                  000072a0    0000003c     driverlib.lib : sys_ctrl.o (.text.NOROM_SysCtrlIdle)
                  000072dc    0000003c     drivers_cc13x2.a : PowerCC26X2_calibrateRCOSC_helpers.c.obj (.text.PowerCC26X2_setTdcClkSrc24M)
                  00007318    0000003c     ti_sysbios_config.o (.text.ti_sysbios_family_arm_m3_Hwi_setPriority)
                  00007354    0000003c     ti_sysbios_config.o (.text.ti_sysbios_knl_Task_restoreHwi)
                  00007390    00000038     ti_drivers_config.o (.text.Board_wakeUpExtFlash)
                  000073c8    00000038     drivers_cc13x2.a : PowerCC26X2_helpers.c.obj (.text.PowerCC26X2_oscDisableQualifiers)
                  00007400    00000038     rf_multiMode_cc13x2.a : rf_patch_cpe_multi_protocol.c.cc13x2.ticlang.o (.text.rf_patch_cpe_multi_protocol)
                  00007438    00000038     ti_sysbios_config.o (.text.ti_sysbios_runtime_Startup_exec)
                  00007470    00000038     libc.a : autoinit.c.obj (.text:__TI_auto_init_nobinit_nopinit)
                  000074a8    00000036     ti_sysbios_config.o (.text.BIOS_rtsUnlock)
                  000074de    00000036     ti_sysbios_config.o (.text.SemaphoreP_pend)
                  00007514    00000036     ti_sysbios_config.o (.text.ti_sysbios_knl_Swi_construct2)
                  0000754a    00000002     --HOLE-- [fill = 0]
                  0000754c    00000034     drivers_cc13x2.a : PowerCC26X2.c.obj (.text.Power_releaseConstraint)
                  00007580    00000034     rf_multiMode_cc13x2.a : RFCC26X2_multiMode.c.cc13x2.ticlang.o (.text.RF_powerConstraintRelease)
                  000075b4    00000034     libc.a : rand.c.obj (.text.rand)
                  000075e8    00000034     ti_sysbios_config.o (.text.ti_sysbios_family_arm_cc26xx_Timer_getMaxTicks)
                  0000761c    00000034     ti_sysbios_config.o (.text.ti_sysbios_knl_Queue_put)
                  00007650    00000034     sysbios.a : boot_cortex_m.obj (.text:_c_int00)
                  00007684    00000032     ti_sysbios_config.o (.text.ti_sysbios_knl_Semaphore_create)
                  000076b6    00000002     --HOLE-- [fill = 0]
                  000076b8    00000030     drivers_cc13x2.a : PowerCC26X2.c.obj (.text.Power_setConstraint)
                  000076e8    00000030     rf_multiMode_cc13x2.a : RFCC26X2_multiMode.c.cc13x2.ticlang.o (.text.RF_checkCmdFsError)
                  00007718    00000030     drivers_cc13x2.a : PowerCC26X2.c.obj (.text.notify)
                  00007748    00000030     ti_sysbios_config.o (.text.ti_sysbios_family_arm_m3_Hwi_plug)
                  00007778    00000030     ti_sysbios_config.o (.text.ti_sysbios_heaps_HeapMem_free)
                  000077a8    00000030     ti_sysbios_config.o (.text.ti_sysbios_knl_Clock_construct)
                  000077d8    00000030     ti_sysbios_config.o (.text.ti_sysbios_knl_Idle_run)
                  00007808    0000002e     driverlib.lib : chipinfo.o (.text.NOROM_ThisLibraryIsFor_CC13x2_CC26x2_HwRev20AndLater_HaltIfViolated)
                  00007836    0000002e     rf_multiMode_cc13x2.a : RFCC26X2_multiMode.c.cc13x2.ticlang.o (.text.RF_calculateDeltaTimeUs)
                  00007864    0000002e     ti_sysbios_config.o (.text._pthread_delete)
                  00007892    0000002e     ti_sysbios_config.o (.text.ti_sysbios_family_arm_m3_Hwi_initStack)
                  000078c0    0000002e     ti_sysbios_config.o (.text.ti_sysbios_gates_GateMutex_Instance_init)
                  000078ee    0000002c     ti_sysbios_config.o (.text.BIOS_registerRTSLock)
                  0000791a    0000002c     ti_sysbios_config.o (.text.BIOS_removeRTSLock)
                  00007946    0000002c     EasyLink.o (.text.EasyLink_Params_init)
                  00007972    00000002     --HOLE-- [fill = 0]
                  00007974    0000002c     rf_multiMode_cc13x2.a : RFCC26X2_multiMode.c.cc13x2.ticlang.o (.text.RF_executeDirectImmediateCmd)
                  000079a0    0000002c     ti_sysbios_config.o (.text.ti_sysbios_knl_Semaphore_construct)
                  000079cc    0000002c     ti_sysbios_config.o (.text.ti_sysbios_runtime_Memory_free)
                  000079f8    0000002a     driverlib.lib : osc.o (.text.NOROM_OSCHF_TurnOnXosc)
                  00007a22    0000002a     ti_sysbios_config.o (.text.SemaphoreP_constructBinary)
                  00007a4c    0000002a     ti_sysbios_config.o (.text.ti_sysbios_knl_Clock_initI)
                  00007a76    0000002a     ti_sysbios_config.o (.text.ti_sysbios_knl_Task_enter)
                  00007aa0    00000028     drivers_cc13x2.a : List.c.obj (.text.List_remove)
                  00007ac8    00000028     driverlib.lib : chipinfo.o (.text.NOROM_ChipInfo_GetChipFamily)
                  00007af0    00000028     rf_multiMode_cc13x2.a : RFCC26X2_multiMode.c.cc13x2.ticlang.o (.text.RF_cmdStoreEvents)
                  00007b18    00000028     sysbios.a : Hwi_asm_gnu.obj (.text.ti_sysbios_family_arm_m3_Hwi_excHandlerAsm)
                  00007b40    00000028     ti_sysbios_config.o (.text.ti_sysbios_gates_GateMutex_construct)
                  00007b68    00000028     ti_sysbios_config.o (.text.ti_sysbios_knl_Queue_enqueue)
                  00007b90    00000028     ti_sysbios_config.o (.text.ti_sysbios_knl_Swi_or)
                  00007bb8    00000028     ti_sysbios_config.o (.text.ti_sysbios_knl_TaskSupport_checkStack)
                  00007be0    00000028     sysbios.a : TaskSupport_asm_gnu.obj (.text.ti_sysbios_knl_TaskSupport_swap)
                  00007c08    00000028     ti_sysbios_config.o (.text.ti_sysbios_runtime_System_init)
                  00007c30    00000026     drivers_cc13x2.a : List.c.obj (.text.List_insert)
                  00007c56    00000026                      : List.c.obj (.text.List_putHead)
                  00007c7c    00000026     rf_multiMode_cc13x2.a : RFCC26X2_multiMode.c.cc13x2.ticlang.o (.text.RF_runCmd)
                  00007ca2    00000026                           : RFCC26X2_multiMode.c.cc13x2.ticlang.o (.text.RF_runScheduleCmd)
                  00007cc8    00000026     ti_sysbios_config.o (.text.ti_sysbios_family_arm_m3_Hwi_getHandle)
                  00007cee    00000026     ti_sysbios_config.o (.text.ti_sysbios_knl_Swi_destruct)
                  00007d14    00000026     ti_sysbios_config.o (.text.ti_sysbios_knl_Task_allBlockedFunction)
                  00007d3a    00000026     ti_sysbios_config.o (.text.ti_sysbios_knl_Task_delete)
                  00007d60    00000026     ti_sysbios_config.o (.text.ti_sysbios_knl_Task_destruct)
                  00007d86    00000026     ti_sysbios_config.o (.text.ti_sysbios_runtime_Error_init)
                  00007dac    00000024     ti_sysbios_config.o (.text.HwiP_setFunc)
                  00007dd0    00000024     drivers_cc13x2.a : List.c.obj (.text.List_put)
                  00007df4    00000024                      : PowerCC26X2_calibrateRCOSC_helpers.c.obj (.text.PowerCC26X2_writeCtrim)
                  00007e18    00000024                      : PowerCC26X2_calibrateRCOSC_helpers.c.obj (.text.PowerCC26X2_writeCtrimFract)
                  00007e3c    00000024                      : PowerCC26X2_calibrateRCOSC_helpers.c.obj (.text.PowerCC26X2_writeCtrimFractEn)
                  00007e60    00000024                      : PowerCC26X2_calibrateRCOSC_helpers.c.obj (.text.PowerCC26X2_writeRtrim)
                  00007e84    00000024                      : PowerCC26X2.c.obj (.text.Power_registerNotify)
                  00007ea8    00000024     rf_multiMode_cc13x2.a : RFCC26X2_multiMode.c.cc13x2.ticlang.o (.text.RF_clkPowerUp)
                  00007ecc    00000024                           : RFCC26X2_multiMode.c.cc13x2.ticlang.o (.text.RF_hwiCpe0ChangePhy)
                  00007ef0    00000024                           : RFCC26X2_multiMode.c.cc13x2.ticlang.o (.text.RF_isStateTransitionAllowed)
                  00007f14    00000024                           : RFCC26X2_multiMode.c.cc13x2.ticlang.o (.text.RF_searchAndReplacePAOverride)
                  00007f38    00000024     ti_sysbios_config.o (.text.ti_sysbios_family_arm_cc26xx_Timer_Params_init)
                  00007f5c    00000024     ti_sysbios_config.o (.text.ti_sysbios_knl_Task_Params_init)
                  00007f80    00000022     ti_sysbios_config.o (.text.BIOS_setThreadType)
                  00007fa2    00000022     drivers_cc13x2.a : List.c.obj (.text.List_get)
                  00007fc4    00000022     rf_multiMode_cc13x2.a : RFCC26X2_multiMode.c.cc13x2.ticlang.o (.text.RF_queueEnd)
                  00007fe6    00000022     ti_sysbios_config.o (.text.ti_sysbios_gates_GateMutex_leave)
                  00008008    00000022     ti_sysbios_config.o (.text.ti_sysbios_heaps_HeapMem_restore)
                  0000802a    00000022     ti_sysbios_config.o (.text.ti_sysbios_knl_Clock_getTicks)
                  0000804c    00000022     ti_sysbios_config.o (.text.ti_sysbios_knl_Clock_scheduleNextTick)
                  0000806e    00000022     ti_sysbios_config.o (.text.ti_sysbios_knl_Queue_dequeue)
                  00008090    00000022     ti_sysbios_config.o (.text.ti_sysbios_knl_Semaphore_destruct)
                  000080b2    00000002     --HOLE-- [fill = 0]
                  000080b4    00000020     rf_multiMode_cc13x2.a : rfc.c.cc13x2.ticlang.o (.text.NOROM_RFCDoorbellSendTo)
                  000080d4    00000020                           : rfc.c.cc13x2.ticlang.o (.text.NOROM_RFCOverrideSearch)
                  000080f4    00000020     drivers_cc13x2.a : PowerCC26X2_helpers.c.obj (.text.PowerCC26X2_disableTCXOQual)
                  00008114    00000020                      : PowerCC26X2_helpers.c.obj (.text.PowerCC26X2_enableTCXOQual)
                  00008134    00000020     ti_sysbios_config.o (.text.PowerCC26XX_schedulerDisable)
                  00008154    00000020     ti_sysbios_config.o (.text.PowerCC26XX_schedulerRestore)
                  00008174    00000020     drivers_cc13x2.a : PowerCC26X2.c.obj (.text.Power_unregisterNotify)
                  00008194    00000020     rf_multiMode_cc13x2.a : RFCC26X2_multiMode.c.cc13x2.ticlang.o (.text.RF_cmdAlloc)
                  000081b4    00000020                           : RFCC26X2_multiMode.c.cc13x2.ticlang.o (.text.RF_invokeGlobalCallback)
                  000081d4    00000020                           : RFCC26X2_multiMode.c.cc13x2.ticlang.o (.text.RF_ratIsRunning)
                  000081f4    00000020     ti_sysbios_config.o (.text.ti_sysbios_family_arm_cc26xx_Timer_postInit)
                  00008214    00000020     ti_sysbios_config.o (.text.ti_sysbios_family_arm_m3_Hwi_excHandler)
                  00008234    00000020     ti_sysbios_config.o (.text.ti_sysbios_family_arm_m3_Hwi_post)
                  00008254    00000020     ti_sysbios_config.o (.text.ti_sysbios_knl_ClockSupport_getCurrentTick)
                  00008274    0000001e     ti_sysbios_config.o (.text.SwiP_Params_init)
                  00008292    0000001e     sysbios.a : Hwi_asm_switch_gnu.obj (.text.ti_sysbios_family_arm_m3_Hwi_switchAndRunFunc)
                  000082b0    0000001e     ti_sysbios_config.o (.text.ti_sysbios_family_arm_m3_Hwi_switchFromBootStack)
                  000082ce    0000001e     ti_sysbios_config.o (.text.ti_sysbios_knl_Task_unblock)
                  000082ec    0000001c     ti_sysbios_config.o (.text.HwiP_Params_init)
                  00008308    0000001c     drivers_cc13x2.a : PowerCC26X2.c.obj (.text.Power_getTransitionLatency)
                  00008324    0000001c     rf_multiMode_cc13x2.a : RFCC26X2_multiMode.c.cc13x2.ticlang.o (.text.RF_clkInactivityCallback)
                  00008340    0000001c                           : RFCC26X2_multiMode.c.cc13x2.ticlang.o (.text.RF_getPAOverrideOffsetAndValue)
                  0000835c    0000001c                           : RFCC26X2_multiMode.c.cc13x2.ticlang.o (.text.RF_powerConstraintSet)
                  00008378    0000001c                           : RFCC26X2_multiMode.c.cc13x2.ticlang.o (.text.RF_swiFsm)
                  00008394    0000001c     ti_sysbios_config.o (.text.ti_sysbios_family_arm_cc26xx_Timer_dynamicStub)
                  000083b0    0000001c     ti_sysbios_config.o (.text.ti_sysbios_family_arm_m3_Hwi_Params_init)
                  000083cc    0000001c     ti_sysbios_config.o (.text.ti_sysbios_knl_Clock_Instance_finalize)
                  000083e8    0000001c     ti_sysbios_config.o (.text.ti_sysbios_knl_Clock_enqueueI)
                  00008404    0000001c     ti_sysbios_config.o (.text.ti_sysbios_knl_Clock_start)
                  00008420    0000001c     ti_sysbios_config.o (.text.ti_sysbios_knl_Queue_remove)
                  0000843c    0000001c     ti_sysbios_config.o (.text.ti_sysbios_knl_Swi_Params_init)
                  00008458    0000001c     ti_sysbios_config.o (.text.ti_sysbios_knl_Swi_disable)
                  00008474    0000001c     ti_sysbios_config.o (.text.ti_sysbios_knl_Task_disable)
                  00008490    0000001a     ti_sysbios_config.o (.text.BIOS_exitFunc)
                  000084aa    0000001a     EasyLink.o (.text.genActivityTableValue)
                  000084c4    0000001a     ti_sysbios_config.o (.text.ti_sysbios_knl_Semaphore_Instance_finalize)
                  000084de    00000018     ti_sysbios_config.o (.text.BIOS_exit)
                  000084f6    00000002     --HOLE-- [fill = 0]
                  000084f8    00000018     drivers_cc13x2.a : GPIOCC26XX.c.obj (.text.GPIO_disableInt)
                  00008510    00000018                      : PowerCC26X2.c.obj (.text.PowerCC26XX_calibrate)
                  00008528    00000018                      : PowerCC26X2.c.obj (.text.Power_idleFunc)
                  00008540    00000018     rf_multiMode_cc13x2.a : RFCC26X2_multiMode.c.cc13x2.ticlang.o (.text.RF_ScheduleCmdParams_init)
                  00008558    00000018                           : RFCC26X2_multiMode.c.cc13x2.ticlang.o (.text.RF_cancelCmd)
                  00008570    00000018                           : RFCC26X2_multiMode.c.cc13x2.ticlang.o (.text.RF_restartClockTimeout)
                  00008588    00000018     ti_sysbios_config.o (.text.ti_sysbios_family_arm_cc26xx_Timer_getCount64)
                  000085a0    00000018     ti_sysbios_config.o (.text.ti_sysbios_family_arm_m3_Hwi_setFunc)
                  000085b8    00000018     ti_sysbios_config.o (.text.ti_sysbios_knl_ClockSupport_setNextTick)
                  000085d0    00000018     sysbios.a : TaskSupport_asm_gnu.obj (.text.ti_sysbios_knl_TaskSupport_glue)
                  000085e8    00000018     ti_sysbios_config.o (.text.ti_sysbios_runtime_System_abort)
                  00008600    00000016     ti_sysbios_config.o (.text.ClockP_Params_init)
                  00008616    00000016     drivers_cc13x2.a : List.c.obj (.text.List_clearList)
                  0000862c    00000016     ti_sysbios_config.o (.text.ti_sysbios_family_arm_m3_Hwi_enable)
                  00008642    00000016     ti_sysbios_config.o (.text.ti_sysbios_knl_Intrinsics_maxbit)
                  00008658    00000016     ti_sysbios_config.o (.text.ti_sysbios_knl_Queue_construct)
                  0000866e    00000016     ti_sysbios_config.o (.text.ti_sysbios_knl_Queue_empty)
                  00008684    00000016     ti_sysbios_config.o (.text.ti_sysbios_runtime_System_exit)
                  0000869a    00000014     ti_drivers_config.o (.text.Board_init)
                  000086ae    00000014     ti_sysbios_config.o (.text.ClockP_setTimeout)
                  000086c2    00000002     --HOLE-- [fill = 0]
                  000086c4    00000014     drivers_cc13x2.a : GPIOCC26XX.c.obj (.text.GPIO_toggle)
                  000086d8    00000014     rf_multiMode_cc13x2.a : RFCC26X2_multiMode.c.cc13x2.ticlang.o (.text.RF_dbellSyncOnAck)
                  000086ec    00000014     ti_sysbios_config.o (.text.SwiP_or)
                  00008700    00000014     libc.a : args_main.c.obj (.text._args_main)
                  00008714    00000014     ti_sysbios_config.o (.text.ti_sysbios_family_arm_cc26xx_TimestampProvider_init)
                  00008728    00000014     ti_sysbios_config.o (.text.ti_sysbios_family_arm_m3_Hwi_disable)
                  0000873c    00000014     ti_sysbios_config.o (.text.ti_sysbios_knl_Swi_Instance_finalize)
                  00008750    00000014     libclang_rt.builtins.a : aeabi_memset.S.obj (.text)
                  00008764    00000014                            : aeabi_uldivmod.S.obj (.text)
                  00008778    00000012     ti_sysbios_config.o (.text.ti_sysbios_family_arm_m3_Hwi_destruct)
                  0000878a    00000012     ti_sysbios_config.o (.text.ti_sysbios_family_arm_m3_Hwi_doSwiRestore)
                  0000879c    00000012     ti_sysbios_config.o (.text.ti_sysbios_family_arm_m3_Hwi_doTaskRestore)
                  000087ae    00000012     ti_sysbios_config.o (.text.ti_sysbios_heaps_HeapMem_Params_init)
                  000087c0    00000012     ti_sysbios_config.o (.text.ti_sysbios_heaps_HeapMem_init)
                  000087d2    00000012     ti_sysbios_config.o (.text.ti_sysbios_knl_Clock_Params_init)
                  000087e4    00000012     ti_sysbios_config.o (.text.ti_sysbios_knl_Clock_tick)
                  000087f6    00000012     ti_sysbios_config.o (.text.ti_sysbios_knl_Queue_Instance_init)
                  00008808    00000012     ti_sysbios_config.o (.text.ti_sysbios_knl_Semaphore_Params_init)
                  0000881a    00000012     libc.a : memcpy_t2.S.obj (.text:TI_memcpy_small)
                  0000882c    00000010     ti_sysbios_config.o (.text.BIOS_start)
                  0000883c    00000010     EasyLink.o (.text.ChipInfo_ChipFamilyIs_CC13x2_CC26x2)
                  0000884c    00000010     EasyLink.o (.text.ChipInfo_ChipFamilyIs_CC13x2x7_CC26x2x7)
                  0000885c    00000010     EasyLink.o (.text.ChipInfo_ChipFamilyIs_CC26x0R2)
                  0000886c    00000010     ti_sysbios_config.o (.text.ClockP_destruct)
                  0000887c    00000010     ti_sysbios_config.o (.text.ClockP_getTimeout)
                  0000888c    00000010     ti_sysbios_config.o (.text.ClockP_isActive)
                  0000889c    00000010     ti_sysbios_config.o (.text.ClockP_start)
                  000088ac    00000010     ti_sysbios_config.o (.text.ClockP_stop)
                  000088bc    00000010     drivers_cc13x2.a : GPIOCC26XX.c.obj (.text.GPIO_write)
                  000088cc    00000010     ti_sysbios_config.o (.text.HwiP_destruct)
                  000088dc    00000010     ti_sysbios_config.o (.text.HwiP_disable)
                  000088ec    00000010     ti_sysbios_config.o (.text.HwiP_enableInterrupt)
                  000088fc    00000010     ti_sysbios_config.o (.text.HwiP_post)
                  0000890c    00000010     ti_sysbios_config.o (.text.HwiP_restore)
                  0000891c    00000010     rf_multiMode_cc13x2.a : rfc.c.cc13x2.ticlang.o (.text.NOROM_RFCCpeIntGetAndClear)
                  0000892c    00000010                           : rfc.c.cc13x2.ticlang.o (.text.NOROM_RFCHwIntGetAndClear)
                  0000893c    00000010                           : RFCC26X2_multiMode.c.cc13x2.ticlang.o (.text.OUTLINED_FUNCTION_1)
                  0000894c    00000010     drivers_cc13x2.a : PowerCC26X2_helpers.c.obj (.text.PowerCC26X2_oscCtlClearXtal)
                  0000895c    00000010                      : PowerCC26X2_helpers.c.obj (.text.PowerCC26X2_prcmEnableCacheRetention)
                  0000896c    00000010                      : PowerCC26X2_calibrateRCOSC_helpers.c.obj (.text.PowerCC26X2_readCtrim)
                  0000897c    00000010                      : PowerCC26X2_calibrateRCOSC_helpers.c.obj (.text.PowerCC26X2_readCtrimFract)
                  0000898c    00000010                      : PowerCC26X2_calibrateRCOSC_helpers.c.obj (.text.PowerCC26X2_readRtrim)
                  0000899c    00000010                      : PowerCC26X2_helpers.c.obj (.text.PowerCC26X2_switchToTCXO)
                  000089ac    00000010     ti_sysbios_config.o (.text.SemaphoreP_destruct)
                  000089bc    00000010     ti_sysbios_config.o (.text.SemaphoreP_post)
                  000089cc    00000010     ti_sysbios_config.o (.text.SwiP_destruct)
                  000089dc    00000010     ti_sysbios_config.o (.text.SwiP_disable)
                  000089ec    00000010     ti_sysbios_config.o (.text.SwiP_getTrigger)
                  000089fc    00000010     ti_sysbios_config.o (.text.SwiP_restore)
                  00008a0c    00000010     ti_sysbios_config.o (.text.SysCtrlAonUpdate)
                  00008a1c    00000010     ti_sysbios_config.o (.text.ti_sysbios_family_arm_cc26xx_Timer_setPeriod)
                  00008a2c    00000010     ti_sysbios_config.o (.text.ti_sysbios_knl_ClockSupport_getMaxTicks)
                  00008a3c    00000010     ti_sysbios_config.o (.text.ti_sysbios_knl_Clock_destruct)
                  00008a4c    00000010     ti_sysbios_config.o (.text.ti_sysbios_knl_Clock_isActive)
                  00008a5c    00000010     ti_sysbios_config.o (.text.ti_sysbios_knl_Clock_removeI)
                  00008a6c    00000010     ti_sysbios_config.o (.text.ti_sysbios_knl_Clock_setTimeout)
                  00008a7c    00000010     ti_sysbios_config.o (.text.ti_sysbios_knl_Idle_loop)
                  00008a8c    00000010     ti_sysbios_config.o (.text.ti_sysbios_knl_Queue_destruct)
                  00008a9c    00000010     ti_sysbios_config.o (.text.ti_sysbios_knl_Queue_elemClear)
                  00008aac    00000010     ti_sysbios_config.o (.text.ti_sysbios_knl_Swi_enabled)
                  00008abc    00000010     ti_sysbios_config.o (.text.ti_sysbios_runtime_SystemSupport_abort)
                  00008acc    00000010     ti_sysbios_config.o (.text.ti_sysbios_runtime_SystemSupport_exit)
                  00008adc    00000010     libc.a : copy_zero_init.c.obj (.text:decompress:ZI)
                  00008aec    0000000e     ti_sysbios_config.o (.text.BIOS_linkedWithIncorrectBootLibrary)
                  00008afa    0000000e     EasyLink.o (.text.ChipInfo_ChipFamilyIs_CC26x0)
                  00008b08    0000000e     ti_sysbios_config.o (.text.IntMasterDisable)
                  00008b16    0000000e     ti_sysbios_config.o (.text.IntMasterEnable)
                  00008b24    0000000e     drivers_cc13x2.a : PowerCC26X2.c.obj (.text.OUTLINED_FUNCTION_0)
                  00008b32    0000000e     rf_multiMode_cc13x2.a : RFCC26X2_multiMode.c.cc13x2.ticlang.o (.text.OUTLINED_FUNCTION_0)
                  00008b40    0000000e                           : RFCC26X2_multiMode.c.cc13x2.ticlang.o (.text.OUTLINED_FUNCTION_3)
                  00008b4e    0000000e     drivers_cc13x2.a : PowerCC26X2.c.obj (.text.switchToTCXO)
                  00008b5c    0000000e     ti_sysbios_config.o (.text.ti_sysbios_family_arm_m3_Hwi_restore)
                  00008b6a    0000000e     ti_sysbios_config.o (.text.ti_sysbios_heaps_HeapMem_isBlocking)
                  00008b78    0000000e     ti_sysbios_config.o (.text.ti_sysbios_knl_Clock_stop)
                  00008b86    0000000e     libc.a : memset_t2.S.obj (.text:TI_memset_small)
                  00008b94    0000000e            : copy_decompress_none.c.obj (.text:decompress:none)
                  00008ba2    0000000c     ti_sysbios_config.o (.text.AONRTCCurrentCompareValueGet)
                  00008bae    0000000c     ti_sysbios_config.o (.text.BIOS_getThreadType)
                  00008bba    0000000c     ti_sysbios_config.o (.text.ClockP_getSystemTickPeriod)
                  00008bc6    0000000c     driverlib.lib : cpu.o (.text.NOROM_CPUcpsid)
                  00008bd2    0000000c                   : cpu.o (.text.NOROM_CPUcpsie)
                  00008bde    00000002     --HOLE-- [fill = 0]
                  00008be0    0000000c     drivers_cc13x2.a : PowerCC26X2_helpers.c.obj (.text.PowerCC26X2_oscClockSourceGet)
                  00008bec    0000000c                      : PowerCC26X2_helpers.c.obj (.text.PowerCC26X2_sysCtrlGetResetSource)
                  00008bf8    0000000c                      : PowerCC26X2_helpers.c.obj (.text.PowerCC26X2_sysCtrlVoltageConditionalControl)
                  00008c04    0000000c                      : PowerCC26X2.c.obj (.text.Power_getConstraintMask)
                  00008c10    0000000c     rf_multiMode_cc13x2.a : RFCC26X2_multiMode.c.cc13x2.ticlang.o (.text.RF_Params_init)
                  00008c1c    0000000c     libc.a : _lock.c.obj (.text._register_lock)
                  00008c28    0000000c            : _lock.c.obj (.text._register_unlock)
                  00008c34    0000000c     ti_sysbios_config.o (.text.ti_sysbios_knl_Queue_head)
                  00008c40    0000000c     ti_sysbios_config.o (.text.ti_sysbios_knl_Queue_next)
                  00008c4c    0000000c     ti_sysbios_config.o (.text.ti_sysbios_knl_Queue_prev)
                  00008c58    0000000c     ti_sysbios_config.o (.text.ti_sysbios_knl_Swi_getTrigger)
                  00008c64    0000000c     ti_sysbios_config.o (.text.ti_sysbios_knl_Swi_postInit)
                  00008c70    0000000c     ti_sysbios_config.o (.text.ti_sysbios_knl_Swi_self)
                  00008c7c    0000000c     ti_sysbios_config.o (.text.ti_sysbios_knl_Task_self)
                  00008c88    0000000a     rf_multiMode_cc13x2.a : RFCC26X2_multiMode.c.cc13x2.ticlang.o (.text.OUTLINED_FUNCTION_5)
                  00008c92    0000000a     drivers_cc13x2.a : PowerCC26X2_helpers.c.obj (.text.PowerCC26X2_sysCtrlStandby)
                  00008c9c    0000000a     ti_sysbios_config.o (.text.ti_sysbios_gates_GateMutex_handle)
                  00008ca6    0000000a     ti_sysbios_config.o (.text.ti_sysbios_knl_Clock_handle)
                  00008cb0    0000000a     ti_sysbios_config.o (.text.ti_sysbios_knl_Queue_struct)
                  00008cba    0000000a     ti_sysbios_config.o (.text.ti_sysbios_knl_Semaphore_handle)
                  00008cc4    0000000a     ti_sysbios_config.o (.text.ti_sysbios_knl_Swi_startup)
                  00008cce    0000000a     ti_sysbios_config.o (.text.ti_sysbios_runtime_Error_check)
                  00008cd8    0000000a     ti_sysbios_config.o (.text.ti_sysbios_runtime_Types_uargToPtr)
                  00008ce2    00000008     ti_sysbios_config.o (.text.Boot_trimDevice)
                  00008cea    00000008     driverlib.lib : cpu.o (.text.NOROM_CPUdelay)
                  00008cf2    00000008     rf_multiMode_cc13x2.a : RFCC26X2_multiMode.c.cc13x2.ticlang.o (.text.OUTLINED_FUNCTION_2)
                  00008cfa    00000008     drivers_cc13x2.a : PowerCC26X2_helpers.c.obj (.text.PowerCC26X2_oschfTrySwitchToXosc)
                  00008d02    00000008     ti_sysbios_config.o (.text.ResetISR)
                  00008d0a    00000008     ti_sysbios_config.o (.text._system_post_cinit)
                  00008d12    00000008     ti_sysbios_config.o (.text._system_pre_init)
                  00008d1a    00000008     ti_sysbios_config.o (.text.ti_sysbios_family_arm_m3_Hwi_startup)
                  00008d22    00000008     ti_sysbios_config.o (.text.ti_sysbios_runtime_Startup_reset)
                  00008d2a    00000008     ti_sysbios_config.o (.text.ti_sysbios_runtime_SysCallback_defaultAbort)
                  00008d32    00000008     ti_sysbios_config.o (.text.ti_sysbios_runtime_SysCallback_defaultExit)
                  00008d3a    00000008     ti_sysbios_config.o (.text.ti_sysbios_runtime_SystemSupport_init)
                  00008d42    00000008     ti_sysbios_config.o (.text.ti_sysbios_runtime_System_exitSpin)
                  00008d4a    00000006     rf_multiMode_cc13x2.a : RFCC26X2_multiMode.c.cc13x2.ticlang.o (.text.OUTLINED_FUNCTION_4)
                  00008d50    00000006                           : RFCC26X2_multiMode.c.cc13x2.ticlang.o (.text.RF_clkReqAccess)
                  00008d56    00000004                           : rfc.c.cc13x2.ticlang.o (.text.NOROM_RFCOverrideUpdate)
                  00008d5a    00000004     ti_sysbios_config.o (.text.PRCMSleep)
                  00008d5e    00000004     drivers_cc13x2.a : PowerCC26X2_helpers.c.obj (.text.PowerCC26X2_oschfSwitchToRcosc)
                  00008d62    00000004                      : PowerCC26X2_helpers.c.obj (.text.PowerCC26X2_sysCtrlIdle)
                  00008d66    00000004                      : PowerCC26X2_helpers.c.obj (.text.PowerCC26X2_turnOnXosc)
                  00008d6a    00000004     rf_multiMode_cc13x2.a : RFCC26X2_multiMode.c.cc13x2.ticlang.o (.text.RF_defaultExecutionPolicy)
                  00008d6e    00000004     drivers_cc13x2.a : PowerCC26X2.c.obj (.text.configureRFCoreClocks)
                  00008d72    00000004                      : PowerCC26X2.c.obj (.text.nopResourceHandler)
                  00008d76    00000004     ti_sysbios_config.o (.text.ti_sysbios_gates_GateMutex_canBlock)
                  00008d7a    00000004     ti_sysbios_config.o (.text.ti_sysbios_knl_TaskSupport_getStackAlignment)
                  00008d7e    00000004     ti_sysbios_config.o (.text.ti_sysbios_runtime_Memory_getMaxDefaultTypeAlign)
                  00008d82    00000004     ti_sysbios_config.o (.text.ti_sysbios_runtime_System_abortSpin)
                  00008d86    00000002     --HOLE-- [fill = 0]
                  00008d88    00000004     libclang_rt.builtins.a : aeabi_memcpy.S.obj (.text)

.rodata    0    00008d8c    00001397     
                  00008d8c    000006e8     rf_multiMode_cc13x2.a : rf_patch_cpe_multi_protocol.c.cc13x2.ticlang.o (.rodata.patchImageMultiProtocol)
                  00009474    000005d0     ti_sysbios_config.o (.rodata.str1.1)
                  00009a44    00000094     ti_sysbios_config.o (.rodata.ti_sysbios_family_arm_m3_Hwi_excHandlerMin.err)
                  00009ad8    0000008d     ti_sysbios_config.o (.rodata.ti_sysbios_heaps_HeapMem_alloc.err)
                  00009b65    00000089     ti_sysbios_config.o (.rodata.ti_sysbios_family_arm_m3_Hwi_Instance_init.err.1)
                  00009bee    00000089     ti_sysbios_config.o (.rodata.ti_sysbios_family_arm_m3_Hwi_excHandlerMin.err.2)
                  00009c77    00000089     ti_sysbios_config.o (.rodata.ti_sysbios_runtime_Memory_alloc.err)
                  00009d00    00000086     ti_sysbios_config.o (.rodata.ti_sysbios_family_arm_m3_Hwi_Instance_init.err)
                  00009d86    00000083     ti_sysbios_config.o (.rodata.ti_sysbios_knl_Task_checkStacks.err.63)
                  00009e09    00000083     ti_sysbios_config.o (.rodata.ti_sysbios_knl_Task_checkStacks.err.64)
                  00009e8c    0000007b     ti_sysbios_config.o (.rodata.ti_sysbios_knl_Task_checkStacks.err.62)
                  00009f07    0000007b     ti_sysbios_config.o (.rodata.ti_sysbios_knl_Task_checkStacks.err)
                  00009f82    00000054     drivers_cc13x2.a : PowerCC26X2.c.obj (.rodata.resourceDB)
                  00009fd6    0000002f     rfEasyLinkTx.o (.rodata.str1.1)
                  0000a005    00000001     ti_easylink_config.o (.rodata.EasyLink_numSupportedPhys)
                  0000a006    00000001     ti_drivers_config.o (.rodata.GPIO_pinLowerBound)
                  0000a007    00000001     ti_drivers_config.o (.rodata.GPIO_pinUpperBound)
                  0000a008    00000024     ti_sysbios_config.o (.rodata.ti_sysbios_knl_Task_Params_default)
                  0000a02c    00000020     rf_multiMode_cc13x2.a : RFCC26X2_multiMode.c.cc13x2.ticlang.o (.rodata.cst32)
                  0000a04c    0000001c     ti_sysbios_config.o (.rodata.ti_sysbios_family_arm_cc26xx_Timer_Params_default)
                  0000a068    00000018     ti_sysbios_config.o (.rodata.ti_sysbios_family_arm_m3_Hwi_Params_default)
                  0000a080    00000014     ti_drivers_config.o (.rodata.PowerCC26X2_config)
                  0000a094    00000014     ti_sysbios_config.o (.rodata.ti_sysbios_knl_Swi_Params_default)
                  0000a0a8    00000010     EasyLink.o (.rodata.EasyLink_defaultParams)
                  0000a0b8    00000010     ti_drivers_config.o (.rodata.GPIO_config)
                  0000a0c8    0000000c     ti_drivers_config.o (.rodata.RFCC26XX_hwAttrs)
                  0000a0d4    0000000c     ti_sysbios_config.o (.rodata.ti_sysbios_heaps_HeapMem_Params_default)
                  0000a0e0    0000000c     ti_sysbios_config.o (.rodata.ti_sysbios_knl_Clock_Params_default)
                  0000a0ec    0000000c     ti_sysbios_config.o (.rodata.ti_sysbios_knl_Semaphore_Params_default)
                  0000a0f8    00000008     rf_multiMode_cc13x2.a : RFCC26X2_multiMode.c.cc13x2.ticlang.o (.rodata..L__const.RF_hwiCpe0Active.activeCmd)
                  0000a100    00000008     driverlib.lib : aux_sysif.o (.rodata.cst4)
                  0000a108    00000008     ti_sysbios_config.o (.rodata.ti_sysbios_knl_Idle_funcList)
                  0000a110    00000004     ti_sysbios_config.o (.rodata.ti_sysbios_family_arm_m3_Hwi_swiTaskKeyAddress)
                  0000a114    00000004     ti_sysbios_config.o (.rodata.ti_sysbios_gates_GateMutex_Params_default)
                  0000a118    00000004     ti_sysbios_config.o (.rodata.ti_sysbios_knl_Clock_tickPeriod)
                  0000a11c    00000004     ti_sysbios_config.o (.rodata.ti_sysbios_knl_Swi_numPriorities)
                  0000a120    00000001     ti_sysbios_config.o (.rodata.ti_sysbios_knl_Clock_tickMode)
                  0000a121    00000001     ti_sysbios_config.o (.rodata.ti_sysbios_knl_Task_checkStackFlag)
                  0000a122    00000001     ti_sysbios_config.o (.rodata.ti_sysbios_knl_Task_initStackFlag)

.args      0    0000a124    00000008     
                  0000a124    00000008     --HOLE-- [fill = 0]

MODULE SUMMARY

       Module                                           code    ro data   rw data
       ------                                           ----    -------   -------
    .\
       rfEasyLinkTx.o                                   578     47        1154   
    +--+------------------------------------------------+-------+---------+---------+
       Total:                                           578     47        1154   
                                                                                 
    .\easylink\
       EasyLink.o                                       3746    16        783    
    +--+------------------------------------------------+-------+---------+---------+
       Total:                                           3746    16        783    
                                                                                 
    .\smartrf_settings\
       ti_radio_config.o                                0       0         292    
    +--+------------------------------------------------+-------+---------+---------+
       Total:                                           0       0         292    
                                                                                 
    .\syscfg\
       ti_sysbios_config.o                              15076   3061      1774   
       ti_drivers_config.o                              314     50        372    
       ti_devices_config.o                              0       88        0      
       ti_easylink_config.o                             0       1         36     
    +--+------------------------------------------------+-------+---------+---------+
       Total:                                           15390   3200      2182   
                                                                                 
    C:/ti/simplelink_cc13xx_cc26xx_sdk_6_20_00_29/kernel/tirtos7/packages/ti/sysbios/lib/ticlang/m4f/sysbios.a
       Hwi_asm_gnu.obj                                  324     0         0      
       Hwi_asm_switch_gnu.obj                           118     0         0      
       TaskSupport_asm_gnu.obj                          64      0         0      
       boot_cortex_m.obj                                52      0         0      
    +--+------------------------------------------------+-------+---------+---------+
       Total:                                           558     0         0      
                                                                                 
    C:/ti/simplelink_cc13xx_cc26xx_sdk_6_20_00_29/source/ti/devices/cc13x2_cc26x2/driverlib/bin/ticlang/driverlib.lib
       osc.o                                            538     0         32     
       sys_ctrl.o                                       432     0         0      
       setup.o                                          392     0         0      
       chipinfo.o                                       338     0         0      
       prcm.o                                           136     0         0      
       aux_sysif.o                                      72      8         0      
       cpu.o                                            32      0         0      
    +--+------------------------------------------------+-------+---------+---------+
       Total:                                           1940    8         32     
                                                                                 
    C:/ti/simplelink_cc13xx_cc26xx_sdk_6_20_00_29/source/ti/drivers/lib/ticlang/m4f/drivers_cc13x2.a
       PowerCC26X2.c.obj                                1822    84        372    
       PowerCC26X2_calibrateRCOSC.c.obj                 836     0         0      
       PowerCC26X2_calibrateRCOSC_helpers.c.obj         436     0         0      
       GPIOCC26X2.c.obj                                 328     0         29     
       PowerCC26X2_helpers.c.obj                        234     0         0      
       List.c.obj                                       208     0         0      
       GPIOCC26XX.c.obj                                 200     0         0      
       GPIO.c.obj                                       60      0         0      
    +--+------------------------------------------------+-------+---------+---------+
       Total:                                           4124    84        401    
                                                                                 
    C:/ti/simplelink_cc13xx_cc26xx_sdk_6_20_00_29/source/ti/drivers/rf/lib/ticlang/m4f/rf_multiMode_cc13x2.a
       RFCC26X2_multiMode.c.cc13x2.ticlang.o            8832    40        1316   
       rf_patch_cpe_multi_protocol.c.cc13x2.ticlang.o   164     1768      1      
       rfc.c.cc13x2.ticlang.o                           268     0         0      
    +--+------------------------------------------------+-------+---------+---------+
       Total:                                           9264    1808      1317   
                                                                                 
    C:\ti\ti-cgt-armllvm_2.1.0.LTS\lib\armv7em-ti-none-eabihf/c/libc.a
       copy_decompress_lzss.c.obj                       106     0         0      
       autoinit.c.obj                                   56      0         0      
       rand.c.obj                                       52      0         4      
       _lock.c.obj                                      26      0         8      
       args_main.c.obj                                  20      0         0      
       memcpy_t2.S.obj                                  18      0         0      
       copy_zero_init.c.obj                             16      0         0      
       copy_decompress_none.c.obj                       14      0         0      
       memset_t2.S.obj                                  14      0         0      
    +--+------------------------------------------------+-------+---------+---------+
       Total:                                           322     0         12     
                                                                                 
    C:\ti\ti-cgt-armllvm_2.1.0.LTS\lib\clang/14.0.5/lib/armv7em-ti-none-eabihf/libclang_rt.builtins.a
       udivmoddi4.S.obj                                 176     0         0      
       aeabi_memset.S.obj                               20      0         0      
       aeabi_uldivmod.S.obj                             20      0         0      
       aeabi_memcpy.S.obj                               4       0         0      
       aeabi_div0.c.obj                                 2       0         0      
    +--+------------------------------------------------+-------+---------+---------+
       Total:                                           222     0         0      
                                                                                 
       Stack:                                           0       0         1024   
       Linker Generated:                                0       440       0      
    +--+------------------------------------------------+-------+---------+---------+
       Grand Total:                                     36144   5603      7197   


LINKER GENERATED COPY TABLES

__TI_cinit_table @ 0000a2d4 records: 2, size/record: 8, table size: 16
	.data: load addr=0000a12c, load size=00000194 bytes, run addr=200051c0, run size=0000065d bytes, compression=lzss
	.bss: load addr=0000a2cc, load size=00000008 bytes, run addr=200040d8, run size=000010e8 bytes, compression=zero_init


LINKER GENERATED HANDLER TABLE

__TI_handler_table @ 0000a2c0 records: 3, size/record: 4, table size: 12
	index: 0, handler: __TI_decompress_lzss
	index: 1, handler: __TI_decompress_none
	index: 2, handler: __TI_zero_init


GLOBAL SYMBOLS: SORTED ALPHABETICALLY BY Name 

address   name                                                               
-------   ----                                                               
20005688  BIOS_Module_state                                                  
00007227  BIOS_atExitFunc                                                    
000084df  BIOS_exit                                                          
00008491  BIOS_exitFunc                                                      
00008baf  BIOS_getThreadType                                                 
20004fc4  BIOS_heapMemObject                                                 
00005a9f  BIOS_init                                                          
00008aed  BIOS_linkedWithIncorrectBootLibrary                                
0000087f  BIOS_nullFunc                                                      
000078ef  BIOS_registerRTSLock                                               
0000791b  BIOS_removeRTSLock                                                 
20005018  BIOS_rtsGate                                                       
00006dbd  BIOS_rtsLock                                                       
000074a9  BIOS_rtsUnlock                                                     
00007f81  BIOS_setThreadType                                                 
0000882d  BIOS_start                                                         
0000669d  BIOS_startFunc                                                     
0000869b  Board_init                                                         
00001017  Board_initHook                                                     
0000522d  Board_sendExtFlashByte                                             
00005b0d  Board_shutDownExtFlash                                             
00007391  Board_wakeUpExtFlash                                               
00008ce3  Boot_trimDevice                                                    
00008601  ClockP_Params_init                                                 
00006175  ClockP_construct                                                   
0000886d  ClockP_destruct                                                    
00008bbb  ClockP_getSystemTickPeriod                                         
0000887d  ClockP_getTimeout                                                  
0000888d  ClockP_isActive                                                    
000086af  ClockP_setTimeout                                                  
0000889d  ClockP_start                                                       
000088ad  ClockP_stop                                                        
00007947  EasyLink_Params_init                                               
00003747  EasyLink_abort                                                     
00007065  EasyLink_getAbsTime                                                
0000003d  EasyLink_init                                                      
0000a005  EasyLink_numSupportedPhys                                          
2000572c  EasyLink_supportedPhys                                             
00000d19  EasyLink_transmitAsync                                             
0000a0b8  GPIO_config                                                        
000084f9  GPIO_disableInt                                                    
00006e01  GPIO_hwiIntFxn                                                     
00003181  GPIO_init                                                          
0000a006  GPIO_pinLowerBound                                                 
0000a007  GPIO_pinUpperBound                                                 
00007265  GPIO_resetConfig                                                   
00004ce5  GPIO_setConfig                                                     
000086c5  GPIO_toggle                                                        
000088bd  GPIO_write                                                         
00004000  HEAPSIZE                                                           
000082ed  HwiP_Params_init                                                   
000062e1  HwiP_construct                                                     
000088cd  HwiP_destruct                                                      
000088dd  HwiP_disable                                                       
000088ed  HwiP_enableInterrupt                                               
000088fd  HwiP_post                                                          
0000890d  HwiP_restore                                                       
00007dad  HwiP_setFunc                                                       
UNDEFED   ITM_flush                                                          
UNDEFED   ITM_restore                                                        
00008617  List_clearList                                                     
00007fa3  List_get                                                           
00007c31  List_insert                                                        
00007dd1  List_put                                                           
00007c57  List_putHead                                                       
00007aa1  List_remove                                                        
00006b3d  NOROM_AUXSYSIFOpModeChange                                         
00008bc7  NOROM_CPUcpsid                                                     
00008bd3  NOROM_CPUcpsie                                                     
00008ceb  NOROM_CPUdelay                                                     
00007ac9  NOROM_ChipInfo_GetChipFamily                                       
00004649  NOROM_ChipInfo_GetChipType                                         
00006799  NOROM_ChipInfo_GetHwRevision                                       
00004179  NOROM_OSCHF_AttemptToSwitchToXosc                                  
0000558d  NOROM_OSCHF_SwitchToRcOscTurnOffXosc                               
000079f9  NOROM_OSCHF_TurnOnXosc                                             
00005605  NOROM_OSC_CapArrayAdjustWorkaround_Boot                            
000068db  NOROM_OSC_HPOSCRelativeFrequencyOffsetGet                          
00006e45  NOROM_PRCMPowerDomainsAllOff                                       
00006e89  NOROM_PRCMPowerDomainsAllOn                                        
000060b9  NOROM_RFCAnaDivTxOverride                                          
0000891d  NOROM_RFCCpeIntGetAndClear                                         
000014af  NOROM_RFCCpePatchReset                                             
000080b5  NOROM_RFCDoorbellSendTo                                            
0000892d  NOROM_RFCHwIntGetAndClear                                          
000080d5  NOROM_RFCOverrideSearch                                            
00008d57  NOROM_RFCOverrideUpdate                                            
00006b85  NOROM_RFCSynthPowerDown                                            
00003c41  NOROM_SetupTrimDevice                                              
000072a1  NOROM_SysCtrlIdle                                                  
000051ad  NOROM_SysCtrlSetRechargeBeforePowerDown                            
00003481  NOROM_SysCtrlStandby                                               
00007809  NOROM_ThisLibraryIsFor_CC13x2_CC26x2_HwRev20AndLater_HaltIfViolated
000070a9  PowerCC26X2_RCOSC_clockFunc                                        
00001bb9  PowerCC26X2_auxISR                                                 
00002e61  PowerCC26X2_calibrate                                              
0000a080  PowerCC26X2_config                                                 
000080f5  PowerCC26X2_disableTCXOQual                                        
00008115  PowerCC26X2_enableTCXOQual                                         
00005ec9  PowerCC26X2_initiateCalibration                                    
200051c0  PowerCC26X2_module                                                 
00008be1  PowerCC26X2_oscClockSourceGet                                      
0000894d  PowerCC26X2_oscCtlClearXtal                                        
000073c9  PowerCC26X2_oscDisableQualifiers                                   
00008d5f  PowerCC26X2_oschfSwitchToRcosc                                     
00008cfb  PowerCC26X2_oschfTrySwitchToXosc                                   
0000895d  PowerCC26X2_prcmEnableCacheRetention                               
0000896d  PowerCC26X2_readCtrim                                              
0000897d  PowerCC26X2_readCtrimFract                                         
0000898d  PowerCC26X2_readRtrim                                              
000070e9  PowerCC26X2_setAclkRefSrc                                          
000072dd  PowerCC26X2_setTdcClkSrc24M                                        
0000899d  PowerCC26X2_switchToTCXO                                           
00008bed  PowerCC26X2_sysCtrlGetResetSource                                  
00008d63  PowerCC26X2_sysCtrlIdle                                            
00008c93  PowerCC26X2_sysCtrlStandby                                         
00008bf9  PowerCC26X2_sysCtrlVoltageConditionalControl                       
00008d67  PowerCC26X2_turnOnXosc                                             
0000567d  PowerCC26X2_updateSubSecInc                                        
00007df5  PowerCC26X2_writeCtrim                                             
00007e19  PowerCC26X2_writeCtrimFract                                        
00007e3d  PowerCC26X2_writeCtrimFractEn                                      
00007e61  PowerCC26X2_writeRtrim                                             
00008511  PowerCC26XX_calibrate                                              
00006ecd  PowerCC26XX_isStableXOSC_HF                                        
00008135  PowerCC26XX_schedulerDisable                                       
00008155  PowerCC26XX_schedulerRestore                                       
00002195  PowerCC26XX_standbyPolicy                                          
200051b0  PowerCC26XX_swiKey                                                 
00006bcd  PowerCC26XX_switchXOSC_HF                                          
200051b4  PowerCC26XX_taskKey                                                
00008c05  Power_getConstraintMask                                            
00008309  Power_getTransitionLatency                                         
00008529  Power_idleFunc                                                     
00002b21  Power_init                                                         
00007e85  Power_registerNotify                                               
0000754d  Power_releaseConstraint                                            
0000422d  Power_releaseDependency                                            
000076b9  Power_setConstraint                                                
000042e1  Power_setDependency                                                
00002039  Power_sleep                                                        
00008175  Power_unregisterNotify                                             
0000a0c8  RFCC26XX_hwAttrs                                                   
200057cc  RFCC26XX_schedulerPolicy                                           
00008c11  RF_Params_init                                                     
00008541  RF_ScheduleCmdParams_init                                          
00008559  RF_cancelCmd                                                       
00002689  RF_close                                                           
20005750  RF_cmdFs                                                           
200056b4  RF_cmdPropRadioDivSetup                                            
20005658  RF_cmdPropRxAdv                                                    
20005768  RF_cmdPropTx                                                       
00008d6b  RF_defaultExecutionPolicy                                          
000048d9  RF_defaultSubmitPolicy                                             
00006745  RF_getCurrentTime                                                  
00001019  RF_open                                                            
0000459d  RF_pendCmd                                                         
00003aa9  RF_postCmd                                                         
00007581  RF_powerConstraintRelease                                          
0000835d  RF_powerConstraintSet                                              
20005780  RF_prop                                                            
00007c7d  RF_runCmd                                                          
00007ca3  RF_runScheduleCmd                                                  
000014b1  RF_scheduleCmd                                                     
00008d03  ResetISR                                                           
00007a23  SemaphoreP_constructBinary                                         
000089ad  SemaphoreP_destruct                                                
000074df  SemaphoreP_pend                                                    
000089bd  SemaphoreP_post                                                    
00008275  SwiP_Params_init                                                   
000052ab  SwiP_construct                                                     
000089cd  SwiP_destruct                                                      
000089dd  SwiP_disable                                                       
000089ed  SwiP_getTrigger                                                    
000086ed  SwiP_or                                                            
000089fd  SwiP_restore                                                       
0000881b  TI_memcpy_small                                                    
00008b87  TI_memset_small                                                    
20014000  __STACK_END                                                        
00000400  __STACK_SIZE                                                       
0000a2d4  __TI_CINIT_Base                                                    
0000a2e4  __TI_CINIT_Limit                                                   
0000a2e4  __TI_CINIT_Warm                                                    
0000a2c0  __TI_Handler_Table_Base                                            
0000a2cc  __TI_Handler_Table_Limit                                           
00007471  __TI_auto_init_nobinit_nopinit                                     
00005d2b  __TI_decompress_lzss                                               
00008b95  __TI_decompress_none                                               
ffffffff  __TI_pprof_out_hndl                                                
ffffffff  __TI_prof_data_size                                                
ffffffff  __TI_prof_data_start                                               
00000000  __TI_static_base__                                                 
00008add  __TI_zero_init                                                     
00002e5f  __aeabi_ldiv0                                                      
0000875d  __aeabi_memclr                                                     
0000875d  __aeabi_memclr4                                                    
0000875d  __aeabi_memclr8                                                    
00008d89  __aeabi_memcpy                                                     
00008d89  __aeabi_memcpy4                                                    
00008d89  __aeabi_memcpy8                                                    
00008751  __aeabi_memset                                                     
00008751  __aeabi_memset4                                                    
00008751  __aeabi_memset8                                                    
00008765  __aeabi_uldivmod                                                   
ffffffff  __binit__                                                          
0000a124  __c_args__                                                         
00057fa8  __ccfg                                                             
UNDEFED   __mpu_init                                                         
200040d8  __primary_heap_end__                                               
200000d8  __primary_heap_start__                                             
20013c00  __stack                                                            
20000000  __start___llvm_prf_bits                                            
20000000  __start___llvm_prf_cnts                                            
20000000  __stop___llvm_prf_bits                                             
20000000  __stop___llvm_prf_cnts                                             
00004391  __udivmoddi4                                                       
00008701  _args_main                                                         
00007651  _c_int00                                                           
20005790  _hposcCoeffs                                                       
200057f0  _lock                                                              
00003077  _nop                                                               
00006f99  _pthread_cleanupFxn                                                
00008c1d  _register_lock                                                     
00008c29  _register_unlock                                                   
00008d0b  _system_post_cinit                                                 
00008d13  _system_pre_init                                                   
200057f4  _unlock                                                            
ffffffff  binit                                                              
0000541f  createTxAdvFromTx                                                  
20004bfc  gpioCallbackFunctions                                              
20005334  gpioPinConfigs                                                     
20004c78  gpioUserArgs                                                       
00006927  main                                                               
200056dc  pOverrides                                                         
000075b5  rand                                                               
00009f82  resourceDB                                                         
00007401  rf_patch_cpe_multi_protocol                                        
200057a0  ti_sysbios_family_arm_cc26xx_Timer_Module_state                    
00007f39  ti_sysbios_family_arm_cc26xx_Timer_Params_init                     
00001a1f  ti_sysbios_family_arm_cc26xx_Timer_construct                       
00008395  ti_sysbios_family_arm_cc26xx_Timer_dynamicStub                     
00008589  ti_sysbios_family_arm_cc26xx_Timer_getCount64                      
00006547  ti_sysbios_family_arm_cc26xx_Timer_getCurrentTick                  
000075e9  ti_sysbios_family_arm_cc26xx_Timer_getMaxTicks                     
00005327  ti_sysbios_family_arm_cc26xx_Timer_periodicStub                    
000081f5  ti_sysbios_family_arm_cc26xx_Timer_postInit                        
0000683d  ti_sysbios_family_arm_cc26xx_Timer_setNextTick                     
00008a1d  ti_sysbios_family_arm_cc26xx_Timer_setPeriod                       
000059bd  ti_sysbios_family_arm_cc26xx_Timer_setThreshold                    
00005dfb  ti_sysbios_family_arm_cc26xx_Timer_start                           
00003c3f  ti_sysbios_family_arm_cc26xx_Timer_startup                         
200051b8  ti_sysbios_family_arm_cc26xx_TimestampProvider_Module_state        
00008715  ti_sysbios_family_arm_cc26xx_TimestampProvider_init                
00005e61  ti_sysbios_family_arm_m3_Hwi_Instance_finalize                     
00003285  ti_sysbios_family_arm_m3_Hwi_Instance_init                         
200055e0  ti_sysbios_family_arm_m3_Hwi_Module_state                          
000083b1  ti_sysbios_family_arm_m3_Hwi_Params_init                           
00006391  ti_sysbios_family_arm_m3_Hwi_construct                             
00004d71  ti_sysbios_family_arm_m3_Hwi_construct2                            
00008779  ti_sysbios_family_arm_m3_Hwi_destruct                              
0000576d  ti_sysbios_family_arm_m3_Hwi_disableInterrupt                      
00002a05  ti_sysbios_family_arm_m3_Hwi_dispatch                              
00005499  ti_sysbios_family_arm_m3_Hwi_dispatchC                             
20004a98  ti_sysbios_family_arm_m3_Hwi_dispatchTable                         
0000878b  ti_sysbios_family_arm_m3_Hwi_doSwiRestore                          
0000879d  ti_sysbios_family_arm_m3_Hwi_doTaskRestore                         
00005a2f  ti_sysbios_family_arm_m3_Hwi_enableInterrupt                       
000012b5  ti_sysbios_family_arm_m3_Hwi_excFillContext                        
00008215  ti_sysbios_family_arm_m3_Hwi_excHandler                            
00007b19  ti_sysbios_family_arm_m3_Hwi_excHandlerAsm                         
00004bc9  ti_sysbios_family_arm_m3_Hwi_excHandlerMin                         
00007cc9  ti_sysbios_family_arm_m3_Hwi_getHandle                             
0000512b  ti_sysbios_family_arm_m3_Hwi_getStackInfo                          
00006c5d  ti_sysbios_family_arm_m3_Hwi_init                                  
00003663  ti_sysbios_family_arm_m3_Hwi_initNVIC                              
00007893  ti_sysbios_family_arm_m3_Hwi_initStack                             
000063e9  ti_sysbios_family_arm_m3_Hwi_initStacks                            
00002adc  ti_sysbios_family_arm_m3_Hwi_interruptsAreDisabledButShouldNotBe   
00002ae1  ti_sysbios_family_arm_m3_Hwi_pendSV                                
00007749  ti_sysbios_family_arm_m3_Hwi_plug                                  
00008235  ti_sysbios_family_arm_m3_Hwi_post                                  
00004f99  ti_sysbios_family_arm_m3_Hwi_postInit                              
20000000  ti_sysbios_family_arm_m3_Hwi_ramVectors                            
00000000  ti_sysbios_family_arm_m3_Hwi_resetVectors                          
00002b04  ti_sysbios_family_arm_m3_Hwi_return                                
000085a1  ti_sysbios_family_arm_m3_Hwi_setFunc                               
00007319  ti_sysbios_family_arm_m3_Hwi_setPriority                           
00008d1b  ti_sysbios_family_arm_m3_Hwi_startup                               
0000a110  ti_sysbios_family_arm_m3_Hwi_swiTaskKeyAddress                     
00008293  ti_sysbios_family_arm_m3_Hwi_switchAndRunFunc                      
000082b1  ti_sysbios_family_arm_m3_Hwi_switchFromBootStack                   
000078c1  ti_sysbios_gates_GateMutex_Instance_init                           
200057d4  ti_sysbios_gates_GateMutex_Module_state                            
00008d77  ti_sysbios_gates_GateMutex_canBlock                                
00007b41  ti_sysbios_gates_GateMutex_construct                               
00007129  ti_sysbios_gates_GateMutex_enter                                   
00007fe7  ti_sysbios_gates_GateMutex_leave                                   
00004b35  ti_sysbios_heaps_HeapMem_Instance_init                             
200057dc  ti_sysbios_heaps_HeapMem_Module_state                              
000087af  ti_sysbios_heaps_HeapMem_Params_init                               
000061d1  ti_sysbios_heaps_HeapMem_alloc                                     
000022d3  ti_sysbios_heaps_HeapMem_allocUnprotected                          
00006441  ti_sysbios_heaps_HeapMem_construct                                 
00007779  ti_sysbios_heaps_HeapMem_free                                      
000038ff  ti_sysbios_heaps_HeapMem_freeUnprotected                           
20005040  ti_sysbios_heaps_HeapMem_gate                                      
00005949  ti_sysbios_heaps_HeapMem_getStats                                  
000087c1  ti_sysbios_heaps_HeapMem_init                                      
00008b6b  ti_sysbios_heaps_HeapMem_isBlocking                                
00008009  ti_sysbios_heaps_HeapMem_restore                                   
00008255  ti_sysbios_knl_ClockSupport_getCurrentTick                         
00008a2d  ti_sysbios_knl_ClockSupport_getMaxTicks                            
00006057  ti_sysbios_knl_ClockSupport_init                                   
000085b9  ti_sysbios_knl_ClockSupport_setNextTick                            
20004d60  ti_sysbios_knl_ClockSupport_timerStruct                            
000083cd  ti_sysbios_knl_Clock_Instance_finalize                             
0000659d  ti_sysbios_knl_Clock_Instance_init                                 
20005418  ti_sysbios_knl_Clock_Module_state                                  
000087d3  ti_sysbios_knl_Clock_Params_init                                   
000077a9  ti_sysbios_knl_Clock_construct                                     
00008a3d  ti_sysbios_knl_Clock_destruct                                      
000083e9  ti_sysbios_knl_Clock_enqueueI                                      
0000802b  ti_sysbios_knl_Clock_getTicks                                      
000071e9  ti_sysbios_knl_Clock_getTicksUntilInterrupt                        
000069c1  ti_sysbios_knl_Clock_getTimeout                                    
00005b7b  ti_sysbios_knl_Clock_init                                          
00007a4d  ti_sysbios_knl_Clock_initI                                         
00008a4d  ti_sysbios_knl_Clock_isActive                                      
00008a5d  ti_sysbios_knl_Clock_removeI                                       
0000804d  ti_sysbios_knl_Clock_scheduleNextTick                              
00008a6d  ti_sysbios_knl_Clock_setTimeout                                    
00008405  ti_sysbios_knl_Clock_start                                         
00003575  ti_sysbios_knl_Clock_startI                                        
00008b79  ti_sysbios_knl_Clock_stop                                          
000087e5  ti_sysbios_knl_Clock_tick                                          
0000a120  ti_sysbios_knl_Clock_tickMode                                      
0000a118  ti_sysbios_knl_Clock_tickPeriod                                    
00003dc9  ti_sysbios_knl_Clock_walkQueueDynamic                              
0000254d  ti_sysbios_knl_Clock_workFuncDynamic                               
0000a108  ti_sysbios_knl_Idle_funcList                                       
00005513  ti_sysbios_knl_Idle_init                                           
2000581a  ti_sysbios_knl_Idle_initDone                                       
00008a7d  ti_sysbios_knl_Idle_loop                                           
000077d9  ti_sysbios_knl_Idle_run                                            
20004798  ti_sysbios_knl_Idle_taskStack                                      
20004dc0  ti_sysbios_knl_Idle_taskStruct                                     
000087f7  ti_sysbios_knl_Queue_Instance_init                                 
00008659  ti_sysbios_knl_Queue_construct                                     
0000806f  ti_sysbios_knl_Queue_dequeue                                       
00008a8d  ti_sysbios_knl_Queue_destruct                                      
00008a9d  ti_sysbios_knl_Queue_elemClear                                     
0000866f  ti_sysbios_knl_Queue_empty                                         
00007b69  ti_sysbios_knl_Queue_enqueue                                       
00008c35  ti_sysbios_knl_Queue_head                                          
00008c41  ti_sysbios_knl_Queue_next                                          
00008c4d  ti_sysbios_knl_Queue_prev                                          
0000761d  ti_sysbios_knl_Queue_put                                           
00008421  ti_sysbios_knl_Queue_remove                                        
000084c5  ti_sysbios_knl_Semaphore_Instance_finalize                         
00006ca5  ti_sysbios_knl_Semaphore_Instance_init                             
200057e4  ti_sysbios_knl_Semaphore_Module_state                              
00008809  ti_sysbios_knl_Semaphore_Params_init                               
000079a1  ti_sysbios_knl_Semaphore_construct                                 
00007685  ti_sysbios_knl_Semaphore_create                                    
00008091  ti_sysbios_knl_Semaphore_destruct                                  
00002d51  ti_sysbios_knl_Semaphore_pend                                      
00007169  ti_sysbios_knl_Semaphore_pendTimeout                               
00004dfd  ti_sysbios_knl_Semaphore_post                                      
0000873d  ti_sysbios_knl_Swi_Instance_finalize                               
000040c1  ti_sysbios_knl_Swi_Instance_init                                   
20005704  ti_sysbios_knl_Swi_Module_state                                    
0000843d  ti_sysbios_knl_Swi_Params_init                                     
00006ceb  ti_sysbios_knl_Swi_construct                                       
00007515  ti_sysbios_knl_Swi_construct2                                      
00007cef  ti_sysbios_knl_Swi_destruct                                        
00008459  ti_sysbios_knl_Swi_disable                                         
00008aad  ti_sysbios_knl_Swi_enabled                                         
00008c59  ti_sysbios_knl_Swi_getTrigger                                      
00006499  ti_sysbios_knl_Swi_init                                            
0000a11c  ti_sysbios_knl_Swi_numPriorities                                   
00007b91  ti_sysbios_knl_Swi_or                                              
00006117  ti_sysbios_knl_Swi_post                                            
00008c65  ti_sysbios_knl_Swi_postInit                                        
20004f64  ti_sysbios_knl_Swi_readyQs                                         
0000688d  ti_sysbios_knl_Swi_restore                                         
00003e89  ti_sysbios_knl_Swi_restoreHwi                                      
000057e5  ti_sysbios_knl_Swi_run                                             
00004c57  ti_sysbios_knl_Swi_runLoop                                         
000053a3  ti_sysbios_knl_Swi_schedule                                        
00008c71  ti_sysbios_knl_Swi_self                                            
00008cc5  ti_sysbios_knl_Swi_startup                                         
00001875  ti_sysbios_knl_TaskSupport_buildTaskStack                          
00007bb9  ti_sysbios_knl_TaskSupport_checkStack                              
00008d7b  ti_sysbios_knl_TaskSupport_getStackAlignment                       
000085d1  ti_sysbios_knl_TaskSupport_glue                                    
000044ef  ti_sysbios_knl_TaskSupport_init                                    
000046f3  ti_sysbios_knl_TaskSupport_start                                   
00007be1  ti_sysbios_knl_TaskSupport_swap                                    
00007bec  ti_sysbios_knl_TaskSupport_swapReturn                              
00002f6d  ti_sysbios_knl_Task_Instance_finalize                              
00001d4d  ti_sysbios_knl_Task_Instance_init                                  
2000561c  ti_sysbios_knl_Task_Module_state                                   
00007f5d  ti_sysbios_knl_Task_Params_init                                    
00007d15  ti_sysbios_knl_Task_allBlockedFunction                             
0000585d  ti_sysbios_knl_Task_blockI                                         
0000a121  ti_sysbios_knl_Task_checkStackFlag                                 
00003823  ti_sysbios_knl_Task_checkStacks                                    
00006af1  ti_sysbios_knl_Task_construct                                      
200051bc  ti_sysbios_knl_Task_defaultStackHeap                               
00007d3b  ti_sysbios_knl_Task_delete                                         
00007d61  ti_sysbios_knl_Task_destruct                                       
00008475  ti_sysbios_knl_Task_disable                                        
00007a77  ti_sysbios_knl_Task_enter                                          
000071a9  ti_sysbios_knl_Task_exit                                           
0000622d  ti_sysbios_knl_Task_init                                           
0000a122  ti_sysbios_knl_Task_initStackFlag                                  
00004005  ti_sysbios_knl_Task_postInit                                       
00006d31  ti_sysbios_knl_Task_processVitalTaskFlag                           
20004f94  ti_sysbios_knl_Task_readyQs                                        
00006fdd  ti_sysbios_knl_Task_restore                                        
00007355  ti_sysbios_knl_Task_restoreHwi                                     
00004795  ti_sysbios_knl_Task_schedule                                       
00008c7d  ti_sysbios_knl_Task_self                                           
000050a7  ti_sysbios_knl_Task_startup                                        
000082cf  ti_sysbios_knl_Task_unblock                                        
00006d77  ti_sysbios_knl_Task_unblockI                                       
00008ccf  ti_sysbios_runtime_Error_check                                     
200057ac  ti_sysbios_runtime_Error_ignore                                    
00007d87  ti_sysbios_runtime_Error_init                                      
00007021  ti_sysbios_runtime_Error_raiseX                                    
00005021  ti_sysbios_runtime_Memory_alloc                                    
2000580c  ti_sysbios_runtime_Memory_defaultHeapInstance                      
000079cd  ti_sysbios_runtime_Memory_free                                     
00008d7f  ti_sysbios_runtime_Memory_getMaxDefaultTypeAlign                   
2000581b  ti_sysbios_runtime_Startup_done                                    
00007439  ti_sysbios_runtime_Startup_exec                                    
00008d23  ti_sysbios_runtime_Startup_reset                                   
00008d2b  ti_sysbios_runtime_SysCallback_defaultAbort                        
00008d33  ti_sysbios_runtime_SysCallback_defaultExit                         
00004837  ti_sysbios_runtime_SysCallback_defaultInit                         
00008abd  ti_sysbios_runtime_SystemSupport_abort                             
00008acd  ti_sysbios_runtime_SystemSupport_exit                              
00008d3b  ti_sysbios_runtime_SystemSupport_init                              
200057b8  ti_sysbios_runtime_System_Module_state                             
000085e9  ti_sysbios_runtime_System_abort                                    
00008d83  ti_sysbios_runtime_System_abortSpin                                
000065f3  ti_sysbios_runtime_System_atexit                                   
200050ec  ti_sysbios_runtime_System_atexitHandlers                           
00008685  ti_sysbios_runtime_System_exit                                     
00008d43  ti_sysbios_runtime_System_exitSpin                                 
00007c09  ti_sysbios_runtime_System_init                                     
00006a0d  ti_sysbios_runtime_System_processAtExit                            
00006a59  txDoneCb                                                           
200054e4  txPowerTable_433_pa13                                              
20004e18  txTask                                                             
00006aa5  txTask_init                                                        


GLOBAL SYMBOLS: SORTED BY Symbol Address 

address   name                                                               
-------   ----                                                               
00000000  __TI_static_base__                                                 
00000000  ti_sysbios_family_arm_m3_Hwi_resetVectors                          
0000003d  EasyLink_init                                                      
00000400  __STACK_SIZE                                                       
0000087f  BIOS_nullFunc                                                      
00000d19  EasyLink_transmitAsync                                             
00001017  Board_initHook                                                     
00001019  RF_open                                                            
000012b5  ti_sysbios_family_arm_m3_Hwi_excFillContext                        
000014af  NOROM_RFCCpePatchReset                                             
000014b1  RF_scheduleCmd                                                     
00001875  ti_sysbios_knl_TaskSupport_buildTaskStack                          
00001a1f  ti_sysbios_family_arm_cc26xx_Timer_construct                       
00001bb9  PowerCC26X2_auxISR                                                 
00001d4d  ti_sysbios_knl_Task_Instance_init                                  
00002039  Power_sleep                                                        
00002195  PowerCC26XX_standbyPolicy                                          
000022d3  ti_sysbios_heaps_HeapMem_allocUnprotected                          
0000254d  ti_sysbios_knl_Clock_workFuncDynamic                               
00002689  RF_close                                                           
00002a05  ti_sysbios_family_arm_m3_Hwi_dispatch                              
00002adc  ti_sysbios_family_arm_m3_Hwi_interruptsAreDisabledButShouldNotBe   
00002ae1  ti_sysbios_family_arm_m3_Hwi_pendSV                                
00002b04  ti_sysbios_family_arm_m3_Hwi_return                                
00002b21  Power_init                                                         
00002d51  ti_sysbios_knl_Semaphore_pend                                      
00002e5f  __aeabi_ldiv0                                                      
00002e61  PowerCC26X2_calibrate                                              
00002f6d  ti_sysbios_knl_Task_Instance_finalize                              
00003077  _nop                                                               
00003181  GPIO_init                                                          
00003285  ti_sysbios_family_arm_m3_Hwi_Instance_init                         
00003481  NOROM_SysCtrlStandby                                               
00003575  ti_sysbios_knl_Clock_startI                                        
00003663  ti_sysbios_family_arm_m3_Hwi_initNVIC                              
00003747  EasyLink_abort                                                     
00003823  ti_sysbios_knl_Task_checkStacks                                    
000038ff  ti_sysbios_heaps_HeapMem_freeUnprotected                           
00003aa9  RF_postCmd                                                         
00003c3f  ti_sysbios_family_arm_cc26xx_Timer_startup                         
00003c41  NOROM_SetupTrimDevice                                              
00003dc9  ti_sysbios_knl_Clock_walkQueueDynamic                              
00003e89  ti_sysbios_knl_Swi_restoreHwi                                      
00004000  HEAPSIZE                                                           
00004005  ti_sysbios_knl_Task_postInit                                       
000040c1  ti_sysbios_knl_Swi_Instance_init                                   
00004179  NOROM_OSCHF_AttemptToSwitchToXosc                                  
0000422d  Power_releaseDependency                                            
000042e1  Power_setDependency                                                
00004391  __udivmoddi4                                                       
000044ef  ti_sysbios_knl_TaskSupport_init                                    
0000459d  RF_pendCmd                                                         
00004649  NOROM_ChipInfo_GetChipType                                         
000046f3  ti_sysbios_knl_TaskSupport_start                                   
00004795  ti_sysbios_knl_Task_schedule                                       
00004837  ti_sysbios_runtime_SysCallback_defaultInit                         
000048d9  RF_defaultSubmitPolicy                                             
00004b35  ti_sysbios_heaps_HeapMem_Instance_init                             
00004bc9  ti_sysbios_family_arm_m3_Hwi_excHandlerMin                         
00004c57  ti_sysbios_knl_Swi_runLoop                                         
00004ce5  GPIO_setConfig                                                     
00004d71  ti_sysbios_family_arm_m3_Hwi_construct2                            
00004dfd  ti_sysbios_knl_Semaphore_post                                      
00004f99  ti_sysbios_family_arm_m3_Hwi_postInit                              
00005021  ti_sysbios_runtime_Memory_alloc                                    
000050a7  ti_sysbios_knl_Task_startup                                        
0000512b  ti_sysbios_family_arm_m3_Hwi_getStackInfo                          
000051ad  NOROM_SysCtrlSetRechargeBeforePowerDown                            
0000522d  Board_sendExtFlashByte                                             
000052ab  SwiP_construct                                                     
00005327  ti_sysbios_family_arm_cc26xx_Timer_periodicStub                    
000053a3  ti_sysbios_knl_Swi_schedule                                        
0000541f  createTxAdvFromTx                                                  
00005499  ti_sysbios_family_arm_m3_Hwi_dispatchC                             
00005513  ti_sysbios_knl_Idle_init                                           
0000558d  NOROM_OSCHF_SwitchToRcOscTurnOffXosc                               
00005605  NOROM_OSC_CapArrayAdjustWorkaround_Boot                            
0000567d  PowerCC26X2_updateSubSecInc                                        
0000576d  ti_sysbios_family_arm_m3_Hwi_disableInterrupt                      
000057e5  ti_sysbios_knl_Swi_run                                             
0000585d  ti_sysbios_knl_Task_blockI                                         
00005949  ti_sysbios_heaps_HeapMem_getStats                                  
000059bd  ti_sysbios_family_arm_cc26xx_Timer_setThreshold                    
00005a2f  ti_sysbios_family_arm_m3_Hwi_enableInterrupt                       
00005a9f  BIOS_init                                                          
00005b0d  Board_shutDownExtFlash                                             
00005b7b  ti_sysbios_knl_Clock_init                                          
00005d2b  __TI_decompress_lzss                                               
00005dfb  ti_sysbios_family_arm_cc26xx_Timer_start                           
00005e61  ti_sysbios_family_arm_m3_Hwi_Instance_finalize                     
00005ec9  PowerCC26X2_initiateCalibration                                    
00006057  ti_sysbios_knl_ClockSupport_init                                   
000060b9  NOROM_RFCAnaDivTxOverride                                          
00006117  ti_sysbios_knl_Swi_post                                            
00006175  ClockP_construct                                                   
000061d1  ti_sysbios_heaps_HeapMem_alloc                                     
0000622d  ti_sysbios_knl_Task_init                                           
000062e1  HwiP_construct                                                     
00006391  ti_sysbios_family_arm_m3_Hwi_construct                             
000063e9  ti_sysbios_family_arm_m3_Hwi_initStacks                            
00006441  ti_sysbios_heaps_HeapMem_construct                                 
00006499  ti_sysbios_knl_Swi_init                                            
00006547  ti_sysbios_family_arm_cc26xx_Timer_getCurrentTick                  
0000659d  ti_sysbios_knl_Clock_Instance_init                                 
000065f3  ti_sysbios_runtime_System_atexit                                   
0000669d  BIOS_startFunc                                                     
00006745  RF_getCurrentTime                                                  
00006799  NOROM_ChipInfo_GetHwRevision                                       
0000683d  ti_sysbios_family_arm_cc26xx_Timer_setNextTick                     
0000688d  ti_sysbios_knl_Swi_restore                                         
000068db  NOROM_OSC_HPOSCRelativeFrequencyOffsetGet                          
00006927  main                                                               
000069c1  ti_sysbios_knl_Clock_getTimeout                                    
00006a0d  ti_sysbios_runtime_System_processAtExit                            
00006a59  txDoneCb                                                           
00006aa5  txTask_init                                                        
00006af1  ti_sysbios_knl_Task_construct                                      
00006b3d  NOROM_AUXSYSIFOpModeChange                                         
00006b85  NOROM_RFCSynthPowerDown                                            
00006bcd  PowerCC26XX_switchXOSC_HF                                          
00006c5d  ti_sysbios_family_arm_m3_Hwi_init                                  
00006ca5  ti_sysbios_knl_Semaphore_Instance_init                             
00006ceb  ti_sysbios_knl_Swi_construct                                       
00006d31  ti_sysbios_knl_Task_processVitalTaskFlag                           
00006d77  ti_sysbios_knl_Task_unblockI                                       
00006dbd  BIOS_rtsLock                                                       
00006e01  GPIO_hwiIntFxn                                                     
00006e45  NOROM_PRCMPowerDomainsAllOff                                       
00006e89  NOROM_PRCMPowerDomainsAllOn                                        
00006ecd  PowerCC26XX_isStableXOSC_HF                                        
00006f99  _pthread_cleanupFxn                                                
00006fdd  ti_sysbios_knl_Task_restore                                        
00007021  ti_sysbios_runtime_Error_raiseX                                    
00007065  EasyLink_getAbsTime                                                
000070a9  PowerCC26X2_RCOSC_clockFunc                                        
000070e9  PowerCC26X2_setAclkRefSrc                                          
00007129  ti_sysbios_gates_GateMutex_enter                                   
00007169  ti_sysbios_knl_Semaphore_pendTimeout                               
000071a9  ti_sysbios_knl_Task_exit                                           
000071e9  ti_sysbios_knl_Clock_getTicksUntilInterrupt                        
00007227  BIOS_atExitFunc                                                    
00007265  GPIO_resetConfig                                                   
000072a1  NOROM_SysCtrlIdle                                                  
000072dd  PowerCC26X2_setTdcClkSrc24M                                        
00007319  ti_sysbios_family_arm_m3_Hwi_setPriority                           
00007355  ti_sysbios_knl_Task_restoreHwi                                     
00007391  Board_wakeUpExtFlash                                               
000073c9  PowerCC26X2_oscDisableQualifiers                                   
00007401  rf_patch_cpe_multi_protocol                                        
00007439  ti_sysbios_runtime_Startup_exec                                    
00007471  __TI_auto_init_nobinit_nopinit                                     
000074a9  BIOS_rtsUnlock                                                     
000074df  SemaphoreP_pend                                                    
00007515  ti_sysbios_knl_Swi_construct2                                      
0000754d  Power_releaseConstraint                                            
00007581  RF_powerConstraintRelease                                          
000075b5  rand                                                               
000075e9  ti_sysbios_family_arm_cc26xx_Timer_getMaxTicks                     
0000761d  ti_sysbios_knl_Queue_put                                           
00007651  _c_int00                                                           
00007685  ti_sysbios_knl_Semaphore_create                                    
000076b9  Power_setConstraint                                                
00007749  ti_sysbios_family_arm_m3_Hwi_plug                                  
00007779  ti_sysbios_heaps_HeapMem_free                                      
000077a9  ti_sysbios_knl_Clock_construct                                     
000077d9  ti_sysbios_knl_Idle_run                                            
00007809  NOROM_ThisLibraryIsFor_CC13x2_CC26x2_HwRev20AndLater_HaltIfViolated
00007893  ti_sysbios_family_arm_m3_Hwi_initStack                             
000078c1  ti_sysbios_gates_GateMutex_Instance_init                           
000078ef  BIOS_registerRTSLock                                               
0000791b  BIOS_removeRTSLock                                                 
00007947  EasyLink_Params_init                                               
000079a1  ti_sysbios_knl_Semaphore_construct                                 
000079cd  ti_sysbios_runtime_Memory_free                                     
000079f9  NOROM_OSCHF_TurnOnXosc                                             
00007a23  SemaphoreP_constructBinary                                         
00007a4d  ti_sysbios_knl_Clock_initI                                         
00007a77  ti_sysbios_knl_Task_enter                                          
00007aa1  List_remove                                                        
00007ac9  NOROM_ChipInfo_GetChipFamily                                       
00007b19  ti_sysbios_family_arm_m3_Hwi_excHandlerAsm                         
00007b41  ti_sysbios_gates_GateMutex_construct                               
00007b69  ti_sysbios_knl_Queue_enqueue                                       
00007b91  ti_sysbios_knl_Swi_or                                              
00007bb9  ti_sysbios_knl_TaskSupport_checkStack                              
00007be1  ti_sysbios_knl_TaskSupport_swap                                    
00007bec  ti_sysbios_knl_TaskSupport_swapReturn                              
00007c09  ti_sysbios_runtime_System_init                                     
00007c31  List_insert                                                        
00007c57  List_putHead                                                       
00007c7d  RF_runCmd                                                          
00007ca3  RF_runScheduleCmd                                                  
00007cc9  ti_sysbios_family_arm_m3_Hwi_getHandle                             
00007cef  ti_sysbios_knl_Swi_destruct                                        
00007d15  ti_sysbios_knl_Task_allBlockedFunction                             
00007d3b  ti_sysbios_knl_Task_delete                                         
00007d61  ti_sysbios_knl_Task_destruct                                       
00007d87  ti_sysbios_runtime_Error_init                                      
00007dad  HwiP_setFunc                                                       
00007dd1  List_put                                                           
00007df5  PowerCC26X2_writeCtrim                                             
00007e19  PowerCC26X2_writeCtrimFract                                        
00007e3d  PowerCC26X2_writeCtrimFractEn                                      
00007e61  PowerCC26X2_writeRtrim                                             
00007e85  Power_registerNotify                                               
00007f39  ti_sysbios_family_arm_cc26xx_Timer_Params_init                     
00007f5d  ti_sysbios_knl_Task_Params_init                                    
00007f81  BIOS_setThreadType                                                 
00007fa3  List_get                                                           
00007fe7  ti_sysbios_gates_GateMutex_leave                                   
00008009  ti_sysbios_heaps_HeapMem_restore                                   
0000802b  ti_sysbios_knl_Clock_getTicks                                      
0000804d  ti_sysbios_knl_Clock_scheduleNextTick                              
0000806f  ti_sysbios_knl_Queue_dequeue                                       
00008091  ti_sysbios_knl_Semaphore_destruct                                  
000080b5  NOROM_RFCDoorbellSendTo                                            
000080d5  NOROM_RFCOverrideSearch                                            
000080f5  PowerCC26X2_disableTCXOQual                                        
00008115  PowerCC26X2_enableTCXOQual                                         
00008135  PowerCC26XX_schedulerDisable                                       
00008155  PowerCC26XX_schedulerRestore                                       
00008175  Power_unregisterNotify                                             
000081f5  ti_sysbios_family_arm_cc26xx_Timer_postInit                        
00008215  ti_sysbios_family_arm_m3_Hwi_excHandler                            
00008235  ti_sysbios_family_arm_m3_Hwi_post                                  
00008255  ti_sysbios_knl_ClockSupport_getCurrentTick                         
00008275  SwiP_Params_init                                                   
00008293  ti_sysbios_family_arm_m3_Hwi_switchAndRunFunc                      
000082b1  ti_sysbios_family_arm_m3_Hwi_switchFromBootStack                   
000082cf  ti_sysbios_knl_Task_unblock                                        
000082ed  HwiP_Params_init                                                   
00008309  Power_getTransitionLatency                                         
0000835d  RF_powerConstraintSet                                              
00008395  ti_sysbios_family_arm_cc26xx_Timer_dynamicStub                     
000083b1  ti_sysbios_family_arm_m3_Hwi_Params_init                           
000083cd  ti_sysbios_knl_Clock_Instance_finalize                             
000083e9  ti_sysbios_knl_Clock_enqueueI                                      
00008405  ti_sysbios_knl_Clock_start                                         
00008421  ti_sysbios_knl_Queue_remove                                        
0000843d  ti_sysbios_knl_Swi_Params_init                                     
00008459  ti_sysbios_knl_Swi_disable                                         
00008475  ti_sysbios_knl_Task_disable                                        
00008491  BIOS_exitFunc                                                      
000084c5  ti_sysbios_knl_Semaphore_Instance_finalize                         
000084df  BIOS_exit                                                          
000084f9  GPIO_disableInt                                                    
00008511  PowerCC26XX_calibrate                                              
00008529  Power_idleFunc                                                     
00008541  RF_ScheduleCmdParams_init                                          
00008559  RF_cancelCmd                                                       
00008589  ti_sysbios_family_arm_cc26xx_Timer_getCount64                      
000085a1  ti_sysbios_family_arm_m3_Hwi_setFunc                               
000085b9  ti_sysbios_knl_ClockSupport_setNextTick                            
000085d1  ti_sysbios_knl_TaskSupport_glue                                    
000085e9  ti_sysbios_runtime_System_abort                                    
00008601  ClockP_Params_init                                                 
00008617  List_clearList                                                     
00008659  ti_sysbios_knl_Queue_construct                                     
0000866f  ti_sysbios_knl_Queue_empty                                         
00008685  ti_sysbios_runtime_System_exit                                     
0000869b  Board_init                                                         
000086af  ClockP_setTimeout                                                  
000086c5  GPIO_toggle                                                        
000086ed  SwiP_or                                                            
00008701  _args_main                                                         
00008715  ti_sysbios_family_arm_cc26xx_TimestampProvider_init                
0000873d  ti_sysbios_knl_Swi_Instance_finalize                               
00008751  __aeabi_memset                                                     
00008751  __aeabi_memset4                                                    
00008751  __aeabi_memset8                                                    
0000875d  __aeabi_memclr                                                     
0000875d  __aeabi_memclr4                                                    
0000875d  __aeabi_memclr8                                                    
00008765  __aeabi_uldivmod                                                   
00008779  ti_sysbios_family_arm_m3_Hwi_destruct                              
0000878b  ti_sysbios_family_arm_m3_Hwi_doSwiRestore                          
0000879d  ti_sysbios_family_arm_m3_Hwi_doTaskRestore                         
000087af  ti_sysbios_heaps_HeapMem_Params_init                               
000087c1  ti_sysbios_heaps_HeapMem_init                                      
000087d3  ti_sysbios_knl_Clock_Params_init                                   
000087e5  ti_sysbios_knl_Clock_tick                                          
000087f7  ti_sysbios_knl_Queue_Instance_init                                 
00008809  ti_sysbios_knl_Semaphore_Params_init                               
0000881b  TI_memcpy_small                                                    
0000882d  BIOS_start                                                         
0000886d  ClockP_destruct                                                    
0000887d  ClockP_getTimeout                                                  
0000888d  ClockP_isActive                                                    
0000889d  ClockP_start                                                       
000088ad  ClockP_stop                                                        
000088bd  GPIO_write                                                         
000088cd  HwiP_destruct                                                      
000088dd  HwiP_disable                                                       
000088ed  HwiP_enableInterrupt                                               
000088fd  HwiP_post                                                          
0000890d  HwiP_restore                                                       
0000891d  NOROM_RFCCpeIntGetAndClear                                         
0000892d  NOROM_RFCHwIntGetAndClear                                          
0000894d  PowerCC26X2_oscCtlClearXtal                                        
0000895d  PowerCC26X2_prcmEnableCacheRetention                               
0000896d  PowerCC26X2_readCtrim                                              
0000897d  PowerCC26X2_readCtrimFract                                         
0000898d  PowerCC26X2_readRtrim                                              
0000899d  PowerCC26X2_switchToTCXO                                           
000089ad  SemaphoreP_destruct                                                
000089bd  SemaphoreP_post                                                    
000089cd  SwiP_destruct                                                      
000089dd  SwiP_disable                                                       
000089ed  SwiP_getTrigger                                                    
000089fd  SwiP_restore                                                       
00008a1d  ti_sysbios_family_arm_cc26xx_Timer_setPeriod                       
00008a2d  ti_sysbios_knl_ClockSupport_getMaxTicks                            
00008a3d  ti_sysbios_knl_Clock_destruct                                      
00008a4d  ti_sysbios_knl_Clock_isActive                                      
00008a5d  ti_sysbios_knl_Clock_removeI                                       
00008a6d  ti_sysbios_knl_Clock_setTimeout                                    
00008a7d  ti_sysbios_knl_Idle_loop                                           
00008a8d  ti_sysbios_knl_Queue_destruct                                      
00008a9d  ti_sysbios_knl_Queue_elemClear                                     
00008aad  ti_sysbios_knl_Swi_enabled                                         
00008abd  ti_sysbios_runtime_SystemSupport_abort                             
00008acd  ti_sysbios_runtime_SystemSupport_exit                              
00008add  __TI_zero_init                                                     
00008aed  BIOS_linkedWithIncorrectBootLibrary                                
00008b6b  ti_sysbios_heaps_HeapMem_isBlocking                                
00008b79  ti_sysbios_knl_Clock_stop                                          
00008b87  TI_memset_small                                                    
00008b95  __TI_decompress_none                                               
00008baf  BIOS_getThreadType                                                 
00008bbb  ClockP_getSystemTickPeriod                                         
00008bc7  NOROM_CPUcpsid                                                     
00008bd3  NOROM_CPUcpsie                                                     
00008be1  PowerCC26X2_oscClockSourceGet                                      
00008bed  PowerCC26X2_sysCtrlGetResetSource                                  
00008bf9  PowerCC26X2_sysCtrlVoltageConditionalControl                       
00008c05  Power_getConstraintMask                                            
00008c11  RF_Params_init                                                     
00008c1d  _register_lock                                                     
00008c29  _register_unlock                                                   
00008c35  ti_sysbios_knl_Queue_head                                          
00008c41  ti_sysbios_knl_Queue_next                                          
00008c4d  ti_sysbios_knl_Queue_prev                                          
00008c59  ti_sysbios_knl_Swi_getTrigger                                      
00008c65  ti_sysbios_knl_Swi_postInit                                        
00008c71  ti_sysbios_knl_Swi_self                                            
00008c7d  ti_sysbios_knl_Task_self                                           
00008c93  PowerCC26X2_sysCtrlStandby                                         
00008cc5  ti_sysbios_knl_Swi_startup                                         
00008ccf  ti_sysbios_runtime_Error_check                                     
00008ce3  Boot_trimDevice                                                    
00008ceb  NOROM_CPUdelay                                                     
00008cfb  PowerCC26X2_oschfTrySwitchToXosc                                   
00008d03  ResetISR                                                           
00008d0b  _system_post_cinit                                                 
00008d13  _system_pre_init                                                   
00008d1b  ti_sysbios_family_arm_m3_Hwi_startup                               
00008d23  ti_sysbios_runtime_Startup_reset                                   
00008d2b  ti_sysbios_runtime_SysCallback_defaultAbort                        
00008d33  ti_sysbios_runtime_SysCallback_defaultExit                         
00008d3b  ti_sysbios_runtime_SystemSupport_init                              
00008d43  ti_sysbios_runtime_System_exitSpin                                 
00008d57  NOROM_RFCOverrideUpdate                                            
00008d5f  PowerCC26X2_oschfSwitchToRcosc                                     
00008d63  PowerCC26X2_sysCtrlIdle                                            
00008d67  PowerCC26X2_turnOnXosc                                             
00008d6b  RF_defaultExecutionPolicy                                          
00008d77  ti_sysbios_gates_GateMutex_canBlock                                
00008d7b  ti_sysbios_knl_TaskSupport_getStackAlignment                       
00008d7f  ti_sysbios_runtime_Memory_getMaxDefaultTypeAlign                   
00008d83  ti_sysbios_runtime_System_abortSpin                                
00008d89  __aeabi_memcpy                                                     
00008d89  __aeabi_memcpy4                                                    
00008d89  __aeabi_memcpy8                                                    
00009f82  resourceDB                                                         
0000a005  EasyLink_numSupportedPhys                                          
0000a006  GPIO_pinLowerBound                                                 
0000a007  GPIO_pinUpperBound                                                 
0000a080  PowerCC26X2_config                                                 
0000a0b8  GPIO_config                                                        
0000a0c8  RFCC26XX_hwAttrs                                                   
0000a108  ti_sysbios_knl_Idle_funcList                                       
0000a110  ti_sysbios_family_arm_m3_Hwi_swiTaskKeyAddress                     
0000a118  ti_sysbios_knl_Clock_tickPeriod                                    
0000a11c  ti_sysbios_knl_Swi_numPriorities                                   
0000a120  ti_sysbios_knl_Clock_tickMode                                      
0000a121  ti_sysbios_knl_Task_checkStackFlag                                 
0000a122  ti_sysbios_knl_Task_initStackFlag                                  
0000a124  __c_args__                                                         
0000a2c0  __TI_Handler_Table_Base                                            
0000a2cc  __TI_Handler_Table_Limit                                           
0000a2d4  __TI_CINIT_Base                                                    
0000a2e4  __TI_CINIT_Limit                                                   
0000a2e4  __TI_CINIT_Warm                                                    
00057fa8  __ccfg                                                             
20000000  __start___llvm_prf_bits                                            
20000000  __start___llvm_prf_cnts                                            
20000000  __stop___llvm_prf_bits                                             
20000000  __stop___llvm_prf_cnts                                             
20000000  ti_sysbios_family_arm_m3_Hwi_ramVectors                            
200000d8  __primary_heap_start__                                             
200040d8  __primary_heap_end__                                               
20004798  ti_sysbios_knl_Idle_taskStack                                      
20004a98  ti_sysbios_family_arm_m3_Hwi_dispatchTable                         
20004bfc  gpioCallbackFunctions                                              
20004c78  gpioUserArgs                                                       
20004d60  ti_sysbios_knl_ClockSupport_timerStruct                            
20004dc0  ti_sysbios_knl_Idle_taskStruct                                     
20004e18  txTask                                                             
20004f64  ti_sysbios_knl_Swi_readyQs                                         
20004f94  ti_sysbios_knl_Task_readyQs                                        
20004fc4  BIOS_heapMemObject                                                 
20005018  BIOS_rtsGate                                                       
20005040  ti_sysbios_heaps_HeapMem_gate                                      
200050ec  ti_sysbios_runtime_System_atexitHandlers                           
200051b0  PowerCC26XX_swiKey                                                 
200051b4  PowerCC26XX_taskKey                                                
200051b8  ti_sysbios_family_arm_cc26xx_TimestampProvider_Module_state        
200051bc  ti_sysbios_knl_Task_defaultStackHeap                               
200051c0  PowerCC26X2_module                                                 
20005334  gpioPinConfigs                                                     
20005418  ti_sysbios_knl_Clock_Module_state                                  
200054e4  txPowerTable_433_pa13                                              
200055e0  ti_sysbios_family_arm_m3_Hwi_Module_state                          
2000561c  ti_sysbios_knl_Task_Module_state                                   
20005658  RF_cmdPropRxAdv                                                    
20005688  BIOS_Module_state                                                  
200056b4  RF_cmdPropRadioDivSetup                                            
200056dc  pOverrides                                                         
20005704  ti_sysbios_knl_Swi_Module_state                                    
2000572c  EasyLink_supportedPhys                                             
20005750  RF_cmdFs                                                           
20005768  RF_cmdPropTx                                                       
20005780  RF_prop                                                            
20005790  _hposcCoeffs                                                       
200057a0  ti_sysbios_family_arm_cc26xx_Timer_Module_state                    
200057ac  ti_sysbios_runtime_Error_ignore                                    
200057b8  ti_sysbios_runtime_System_Module_state                             
200057cc  RFCC26XX_schedulerPolicy                                           
200057d4  ti_sysbios_gates_GateMutex_Module_state                            
200057dc  ti_sysbios_heaps_HeapMem_Module_state                              
200057e4  ti_sysbios_knl_Semaphore_Module_state                              
200057f0  _lock                                                              
200057f4  _unlock                                                            
2000580c  ti_sysbios_runtime_Memory_defaultHeapInstance                      
2000581a  ti_sysbios_knl_Idle_initDone                                       
2000581b  ti_sysbios_runtime_Startup_done                                    
20013c00  __stack                                                            
20014000  __STACK_END                                                        
ffffffff  __TI_pprof_out_hndl                                                
ffffffff  __TI_prof_data_size                                                
ffffffff  __TI_prof_data_start                                               
ffffffff  __binit__                                                          
ffffffff  binit                                                              
UNDEFED   ITM_flush                                                          
UNDEFED   ITM_restore                                                        
UNDEFED   __mpu_init                                                         

[456 symbols]
